:020000020000FC
:040000000C9420003C
:020008000001F5
:100034000C948E220C94B9260C94DF21F894A0E041
:100044002A2EA1E03A2EA1E0AEBFAFEFADBF2CBC8B
:100054000E9422210E947E270E94E05C0C943300BF
:10006400FDCF80E090E0AC014C015C01BC016C016F
:100074007C012C01209210012EBAA8E1B1E0E0E24B
:100084002D92EA95E9F785C2E92FF4EBF491E82F74
:10009400F7FF8190F7FD8590F7FF9190F7FD95901C
:1000A400029677C25ABDE92DF4EBF491E82DF7FFDF
:1000B4005193F7FD0E941A216CC2830C921C69C2F1
:1000C40040FB930C4FB740F92EBA63C240FB931820
:1000D4004FB740F93EBA5DC2E92FF4EBF491E82F33
:1000E400F7FF9190F7FD9590019653C24695052F21
:1000F400000F551F441F4F7D5CC20A0140911E0131
:1001040050911F0100921E0110921F0142C2469598
:10011400680D791D441F2EBA3CC2E92DF4EBF4910D
:10012400E82DF7FF5191F7FD559133C283189208DA
:1001340030C240FB830C4FB740F92EBA2AC240FBB1
:1001440083184FB740F93EBA24C2E92FF4EBF49177
:10015400E82FF7FF8190F7FD859001961AC2469526
:10016400052F06955795441F4F7D23C26894931815
:1001740009F4E8943FC2E92FF4EBF491E82FF7FF78
:10018400A190F7FDA590F7FFB190F7FDB590029609
:1001940000C25ABDEB2DF4EBF491EA2DF7FF519315
:1001A400F7FD0E941A21F5C1A30CB21CF2C140FB59
:1001B400B30C4FB740F92EBAECC140FBB3184FB79C
:1001C40040F93EBAE6C1E92FF4EBF491E82FF7FFCA
:1001D400B190F7FDB5900196DCC14695551F441FBB
:1001E4004F7DE7C1689406C246956A0D7B1D441F86
:1001F4002EBACFC1EB2DF4EBF491EA2DF7FF519118
:10020400F7FD5591C6C1A318B208C3C140FBA30CA6
:100214004FB740F92EBABDC140FBA3184FB740F900
:100224003EBAB7C1E92FF4EBF491E82FF7FFA190A0
:10023400F7FDA5900196ADC146955795441F4F7D96
:10024400B8C141FBF5C1E92FF4EBF491E82FF7FFB6
:100254006191F7FD6591F7FF7191F7FD7591029634
:1002640098C1E92FF4EBF491E82FF7FFA191F7FD82
:10027400A591F7FFB191F7FDB5910296EB2FF4EB41
:10028400F491EA2FF7FF6193F7FF719382C1630D35
:10029400721D7FC140FB730D4FB740F92EBA79C16F
:1002A40040FB73194FB740F93EBA73C1E92FF4EB21
:1002B400F491E82FF7FF7191F7FD7591019669C1EB
:1002C400052F0F70F0990EC00A3045FF08F05A5FF1
:1002D400052F007F0A30332708F030E6530F08F467
:1002E400416004C045FD565040FD5056E52FF5EBE6
:1002F40044914FC141FB7EC14695660F771F441F51
:100304002EBA47C1E92FF4EBF491E82FF7FFA1913E
:10031400F7FDA591F7FFB191F7FDB5910296EB2F8B
:10032400F4EBF491EA2FF7FF6191F7FD6591F7FF84
:100334007191F7FD75912DC1631972092AC140FBB2
:10034400630D4FB740F92EBA24C140FB63194FB770
:1003540040F93EBA1EC1E92FF4EBF491E82FF7FF00
:100364006191F7FD6591019614C1509540623EBAC2
:1003740010C140FB5DC1E92FF4EBF491E82FF7FFC6
:100384004190F7FD4590F7FF5190F7FD5590029687
:1003940000C1E92FF4EBF491E82FF7FFA191F7FDE9
:1003A400A591F7FFB191F7FDB59102965ABDEB2FD8
:1003B400F4EBF491EA2FF7FF5193F7FD0E941A2111
:1003C400E8C0430C521CE5C0E72FF4EBF491E62F90
:1003D400F7FF0191F7FD059140FB030D4FB740F97D
:1003E4002EBAD6C0E72FF4EBF491E62FF7FF019174
:1003F400F7FD059140FB03194FB740F93EBAC8C059
:10040400E92FF4EBF491E82FF7FF0191F7FD059143
:100414000196BEC04F7D2EBA4160BBC040FBEAC00E
:100424004695640D751D441F2EBAB3C0E92FF4EB35
:10043400F491E82FF7FFA191F7FDA591F7FFB19192
:10044400F7FDB5910296EB2FF4EBF491EA2FF7FF49
:100454005191F7FD55919DC0431852089AC040FB35
:10046400530D4FB740F92EBA94C040FB53194FB700
:1004740040F93EBA8EC0E92FF4EBF491E82FF7FF70
:100484005191F7FD5591019684C040FB45F94325F0
:1004940090C07FC0982C7DC09B2C7BC09A2C79C0C7
:1004A400972E77C0962E75C05BD6902E72C0952E6F
:1004B40070C0892C6EC06DC08B2C6BC08A2C69C037
:1004C400872E67C0862E65C04BD6802E62C0852ECF
:1004D40060C0B92C5EC0B82C5CC05BC0BA2C59C0DB
:1004E400B72E57C0B62E55C03BD6B02E52C0B52E2F
:1004F40050C0A92C4EC0A82C4CC0AB2C4AC049C03B
:10050400A72E47C0A62E45C02BD6A02E42C0A52E8E
:1005140040C0792D3EC0782D3CC07B2D3AC07A2D49
:1005240038C037C0762F35C01BD6702F32C0752F18
:1005340030C0692D2EC0682D2CC06B2D2AC06A2DA9
:1005440028C0672F26C025C00BD6602F22C0652F78
:1005540020C0092D1DC0082D1BC00B2D19C00A2D4C
:1005640017C0072F15C0062F13C013C0052F10C0C6
:10057400592D0FC0582D0DC05B2D0BC05A2D09C02D
:10058400572F07C0562F05C0EBD5502F02C001C00E
:10059400DCC5EE27E92FF4EBF491E82FF7FF019087
:1005A400F7FD059097FD06FCE02D0196F5E0099412
:1005B4004FB72EBAEE27E92FF4EBF491E82FF7FFAB
:1005C4000190F7FD059097FD06FCE02D0196F5E0FE
:1005D40009944FB73EBAEE27E92FF4EBF491E82FD4
:1005E400F7FF0190F7FD059097FD06FCE02D0196BD
:1005F400F5E00994E92FF4EBF491E82FF7FFE1918A
:10060400F7FDE59101962EF4E058805892098E0F7B
:10061400921DEE27E92FF4EBF491E82FF7FF0190F8
:10062400F7FD059097FD06FCE02D0196F5E0099491
:10063400E92FF4EBF491E82FF7FFE191F7FDE59151
:1006440001962EF0E058805892098E0F921DEE27E5
:10065400E92FF4EBF491E82FF7FF0190F7FD0590F3
:1006640097FD06FCE02D0196F5E00994E92FF4EBE3
:10067400F491E82FF7FFA191F7FDA591F7FFB19150
:10068400F7FDB59102960EF4CD01EE27E92FF4EBB8
:10069400F491E82FF7FF0190F7FD059097FD06FC14
:1006A400E02D0196F5E00994E92FF4EBF491E82F9D
:1006B400F7FFA191F7FDA591F7FFB191F7FDB59172
:1006C40002960EF0CD01EE27E92FF4EBF491E82F1A
:1006D400F7FF0190F7FD059097FD06FCE02D0196CC
:1006E400F5E00994E92FF4EBF491E82FF7FF01907A
:1006F400F7FD0590F7FF1190F7FD15900296CEF4E3
:10070400D20112972D018ABDEB2FF4EBF491EA2F5D
:10071400F7FF8193F7FD0E941A2111969ABDEB2FE2
:10072400F4EBF491EA2FF7FF9193F7FD0E941A215D
:10073400C001EE27E92FF4EBF491E82FF7FF0190C5
:10074400F7FD059097FD06FCE02D0196F5E0099470
:10075400E92FF4EBF491E82FF7FF0190F7FD0590F2
:10076400F7FF1190F7FD15900296CEF0D201129783
:100774002D018ABDEB2FF4EBF491EA2FF7FF81935F
:10078400F7FD0E941A2111969ABDEB2FF4EBF49118
:10079400EA2FF7FF9193F7FD0E941A21C001EE277B
:1007A400E92FF4EBF491E82FF7FF0190F7FD0590A2
:1007B40097FD06FCE02D0196F5E00994002E122C1D
:1007C400D20112972D018ABDEB2FF4EBF491EA2F9D
:1007D400F7FF8193F7FD0E941A2111969ABDEB2F22
:1007E400F4EBF491EA2FF7FF9193F7FD0E941A219D
:1007F400C001EE27E92FF4EBF491E82FF7FF019005
:10080400F7FD059097FD06FCE02D0196F5E00994AF
:10081400A6F4D201EB2FF4EBF491EA2FF7FF8191C8
:10082400F7FD85911196EB2FF4EBF491EA2FF7FF86
:100834009191F7FD959111962D01EE27E92FF4EB97
:10084400F491E82FF7FF0190F7FD059097FD06FC62
:10085400E02D0196F5E00994A6F0D201EB2FF4EB1C
:10086400F491EA2FF7FF8191F7FD85911196EB2F13
:10087400F4EBF491EA2FF7FF9191F7FD959111961E
:100884002D01EE27E92FF4EBF491E82FF7FF019007
:10089400F7FD059097FD06FCE02D0196F5E009941F
:1008A400E52FF5EB44912EBAEE27E92FF4EBF49102
:1008B400E82FF7FF0190F7FD059097FD06FCE02D6A
:1008C4000196F5E00994E52FF5EB44912EBA4F7D9E
:1008D400EE27E92FF4EBF491E82FF7FF0190F7FDF1
:0E08E400059097FD06FCE02D0196F5E00994C5
:100A0000CACD44CB51CB5BCB5DCB62CB67CB70CB3C
:100A100076CB7FCB84CB8CCB8ECB93CB98CBA1CB1F
:100A2000A7CBABCBB8CBC2CBC4CBC9CBCECBD7CB70
:100A3000DBCBDCCBE1CBE9CBEBCBF0CBF5CBFECB0F
:100A400002CC03CC10CC25CC27CC2CCC31CC3ACC4E
:100A500053CC54CC59CC72CC74CC79CC7ECC87CCD2
:100A60008ACC8BCC98CCAFCCB1CCBECCCBCCD4CCBC
:100A7000D7CCD8CCDDCCF2CCF4CCF9CCFECC07CDA5
:100A80000ACD0ACD0BCD0CCD0DCD0ECD0FCD11CD98
:100A900012CD13CD13CD14CD15CD16CD17CD19CD47
:100AA0001ACD1BCD1CCD1CCD1DCD1ECD1FCD21CDF6
:100AB00022CD23CD24CD25CD25CD26CD27CD29CDA5
:100AC0002ACD2BCD2CCD2DCD2ECD2ECD2FCD31CD54
:100AD00032CD33CD34CD35CD36CD37CD37CD39CD03
:100AE0003ACD3BCD3CCD3DCD3ECD3FCD40CD40CDB3
:100AF00041CD42CD43CD44CD45CD46CD47CD49CD69
:100B00007FC080C081C082C083C084C085C08EC0C9
:100B10008FC091C093C095C097C099C09BC0A5C01D
:100B2000A7C0A8C0A9C0AAC0ABC0ACC0ADC0B6C069
:100B3000B7C0BAC0BDC0C0C0C3C0C6C0C9C0D4C0A1
:100B4000D7C0D8C0D9C0DAC0DBC0DCC0DDC0E6C0C9
:100B5000E7C0E8C0E9C0EAC0EBC0ECC0EDC0F6C039
:100B6000F7C0F8C0F9C0FAC0FBC0FCC0FDC006C1A8
:100B700007C108C109C10AC10BC10CC10DC116C111
:100B800017C118C127C128C136C137C142C14CC1E4
:100B90004DC14EC14FC150C151C152C153C15EC1BF
:100BA0005FC160C16FC170C17DC17EC189C193C188
:100BB00094C195C1B0C1B1C1BEC1BFC1C0C1CCC19A
:100BC000CDC1CEC1DDC1DEC1F4C1F5C100C20AC2D2
:100BD0000BC20CC20EC20FC212C213C214C21EC27A
:100BE0001FC220C22FC230C230C231C23CC246C274
:100BF00047C248C24AC24BC24BC24CC24DC257C286
:100C0000590DD8CC580DD6CC5B0DD4CC5A0DD2CCC6
:100C1000570FD0CC560FCECCE72FF4EBF491E62F44
:100C2000F7FF0191F7FD0591500FC4CC550FC2CCD1
:100C30004695591DBFCC4695581DBCCC46955B1DAD
:100C4000B9CC46955A1DB6CC4695571FB3CC4695A0
:100C5000561FB0CCE72FF4EBF491E62FF7FF01918C
:100C6000F7FD05914695501FA5CC4695551FA2CC82
:100C70005919B1CC5819AFCC5B19ADCC5A19ABCCC2
:100C8000571BA9CC561BA7CCE72FF4EBF491E62F0A
:100C9000F7FF0191F7FD0591501B9DCC551B9BCC97
:100CA00046951894590997CC46951894580993CCB1
:100CB000469518945B098FCC469518945A098BCCAD
:100CC00046951894570B87CC46951894560B83CCB1
:100CD000E72FF4EBF491E62FF7FF0191F7FD059173
:100CE00046951894500B77CC46951894550B73CCB9
:100CF0005921D8CD5821D6CD5B21D4CD5A21D2CD82
:100D00005723D0CD5623CECDE72FF4EBF491E62F29
:100D1000F7FF0191F7FD05915023C4CD5523C2CDB6
:100D20005925D3CD5825D1CD5B25CFCD5A25CDCD55
:100D30005727CBCD5627C9CDE72FF4EBF491E62FFB
:100D4000F7FF0191F7FD05915027BFCD5527BDCD88
:100D50005929BBCD5829B9CD5B29B7CD5A29B5CD75
:100D6000572BB3CD562BB1CDE72FF4EBF491E62FF3
:100D7000F7FF0191F7FD0591502BA7CD562BA5CD7F
:100D8000591529CC581527CC5B1525CC5A1523CCE1
:100D9000571721CC56171FCCE72FF4EBF491E62F11
:100DA000F7FF0191F7FD0591501715CC551713CC9E
:100DB00041FB54CDE52DF4EBF491E42DF7FF819048
:100DC000F7FD8590F7FF9190F7FD9590A2E04A0E10
:100DD000521CE1CB41FB6ACCE92FF4EBF491E82FF4
:100DE000F7FF0191F7FD0591F7FF1191F7FD1591BF
:100DF0000296C801D0CB41FBADCCA2E04A1A520802
:100E0000E52DF4EBF491E42DF7FF8192F7FF919239
:100E1000C2CBE92FF4EBF491E82FF7FF0191F7FD36
:100E200005910196500FC6CB00E0CACC41FBF2CC35
:100E30006894F0CC41FB1CCC0C94B80E41FB54CC14
:100E4000689452CCE92FF4EBF491E82FF7FF01916D
:100E5000F7FD059101964695501FACCB08E0B0CC4C
:100E600040FBFCCCE52DF4EBF491E42DF7FFA190D1
:100E7000F7FDA590F7FFB190F7FDB590A2E04A0EFF
:100E8000521C89CB40FB12CCE92FF4EBF491E82FF4
:100E9000F7FF2191F7FD25910196352F052F0E942F
:100EA000D92079CB40FB56CCA2E04A1A5208E52D56
:100EB000F4EBF491E42DF7FFA192F7FFB1926BCB25
:100EC000E92FF4EBF491E82FF7FF0191F7FD05917D
:100ED0000196501B80CB00E173CC40FB9BCC0401FE
:100EE0008090180190901901109219010092180138
:100EF0000501A0901A01B0901B0110921B010092F5
:100F00001A010B0160911C0170911D0110921D01CD
:100F100000921C0140CB40FBABCBE92FF4EBF491EA
:100F2000E82FF7FF2191F7FD25910196352F0E94BB
:100F30009A20502F30CB40FBD7CB0C947712E92F5F
:100F4000F4EBF491E82FF7FF0191F7FD059101967D
:100F500046951894500B3FCB08E132CC43FB7ECC36
:100F6000E52DF4EBF491E42DF7FF6191F7FD659128
:100F7000F7FF7191F7FD7591A2E04A0E521C0BCB61
:100F800043FB94CBD2010B01EB2FF4EBF491EA2F4E
:100F9000F7FF6191F7FD6591F7FF7191F7FD75918D
:100FA000EB2FF4EBF491EA2FF7FF0192F7FF119288
:100FB000F2CA43FBCFCBA2E04A1A5208E52DF4EB6C
:100FC000F491E42DF7FF6193F7FF7193E4CAE92FE1
:100FD000F4EBF491E82FF7FF0191F7FD05910196ED
:100FE000502360CC00E2ECCB43FB14CC862F972F30
:100FF000D2CA43FB3DCB05015B01B001CCCA43FB28
:1010000073CB0C94921CE92FF4EBF491E82FF7FFCB
:101010000191F7FD05910196502757CC08E2D0CBFE
:1010200042FB1CCCE52DF4EBF491E42DF7FF41914C
:10103000F7FD4591F7FF5191F7FD5591A2E04A0E5A
:10104000521CA9CA42FB32CBA6CA42FB83CBA2E008
:101050004A1A5208E52DF4EBF491E42DF7FF419381
:10106000F7FF519398CAE92FF4EBF491E82FF7FFBB
:101070000191F7FD05910196502B27CC00E3A0CB01
:1010800042FBC8CB462E572E86CA42FBF1CA83CA02
:1010900042FB2ACB0C944B19E92FF4EBF491E82F87
:1010A000F7FF0191F7FD05910196501794CA08E3E7
:1010B00087CB02E0401A5208D0E009911881E52D53
:1010C000F4EBF491E42DF7FF0193F7FF119363CA5A
:1010D000D0E0E52DF4EBF491E42DF7FF0191F7FD5D
:1010E0000591F7FF1191F7FD15910993188302E01F
:1010F000400E521C50CAD0E008801980D201EB2F5C
:10110000F4EBF491EA2FF7FF0191F7FD05910ABC8A
:10111000EB2FF4EBF491EA2FF7FF0192F7FD0E9419
:101120001A2111960883EB2FF4EBF491EA2FF7FFC5
:101130000191F7FD05911ABCEB2FF4EBF491EA2F26
:10114000F7FF1192F7FD0E941A21098324CA0ABDF4
:10115000E72FF4EBF491E62FF7FF0193F7FD0E94E0
:101160001A2119CAE72FF4EBF491E62FF7FF01914A
:10117000F7FD05910895FFC003C107C10BC10FC161
:1011800013C117C11CC120C124C128C12CC130C149
:1011900034C138C13DC141C145C149C14DC151C131
:1011A00055C159C15EC162C167C16CC171C176C10F
:1011B0007BC180C186C18BC18EC191C194C197C1D1
:1011C0009AC19DC1A1C1A4C1A9C1AEC1B3C1B8C1D9
:1011D000BDC1C2C1C8C1CDC1D1C1D5C1D9C1DDC197
:1011E000E1C1E5C1EAC1EEC1F1C1F4C1F7C1FAC183
:1011F000FDC100C204C207C20EC215C21CC223C276
:101200002AC231C239C240C247C24EC255C25CC2B4
:1012100063C26AC272C279C280C287C28EC295C2DC
:101220009CC2A3C2ABC2B2C2B9C2C0C2C7C2CEC204
:10123000D5C2DCC2E4C2EBC2F2C2F9C200C307C32A
:101240000EC315C31DC324C32BC332C339C340C34C
:1012500047C34EC356C35DC364C36BC372C379C374
:1012600080C387C38FC396C39DC3A4C3ABC3B2C39C
:10127000B9C3C0C3C8C3CFC3D1C3D3C3D5C3D7C3F6
:10128000D9C3DBC3DEC3E0C3E2C3E4C3E6C3E8C340
:10129000EAC3ECC3EFC3F1C3F3C3F5C3F7C3F9C3A8
:1012A000FBC3FDC300C402C404C406C408C40AC40A
:1012B0000CC40EC411C413C415C417C419C41BC470
:1012C0001DC41FC422C424C426C428C42AC42CC4D8
:1012D0002EC430C433C435C437C439C43BC43DC440
:1012E0003FC441C444C446C448C44AC44CC44EC4A8
:1012F00050C452C455C457C459C45BC45DC45FC410
:1013000061C463C466C468C46AC46CC46EC470C477
:1013100072C474C477C479C47BC47DC47FC481C4DF
:1013200083C485C488C48AC48CC48EC490C492C447
:1013300094C496C499C49BC49DC49FC4A1C4A3C4AF
:10134000A5C4A7C4AAC4ACC4AEC4B0C4B2C4B4C417
:10135000B6C4B8C4BBC4BDC4BFC4C1C4C3C4C5C47F
:10136000C7C4C9C4CCC4CEC4D0C4D2C4D4C4D6C4E7
:10137000D8C4DAC4DDC497FA990C90F8E92DE5C415
:1013800087FA880C80F8E82DE0C4B7FABB0CB0F8F7
:10139000EB2DDBC4A7FAAA0CA0F8EA2DD6C477FB84
:1013A000770F70F9E72FD1C467FB660F60F9E62F5E
:1013B000CCC4ECD407FB000F00F9E02FBCC457FBF2
:1013C000550F50F9E52FC1C490FA969497F8E92D7E
:1013D000BCC480FA869487F8E82DB7C4B0FAB694F6
:1013E000B7F8EB2DB2C4A0FAA694A7F8EA2DADC4C5
:1013F00070FB769577F9E72FA8C460FB669567F9CF
:10140000E62FA3C4C3D400FB069507F9E02F93C4CD
:1014100050FB569557F9E52F98C4469597FA991CB5
:10142000E92D93C4469587FA881CE82D8EC446950D
:10143000B7FABB1CEB2D89C44695A7FAAA1CEA2D66
:1014400084C4469577FB771FE72F7FC4469567FBDB
:10145000661FE62F7AC49AD4469507FB001FE02F3B
:101460006AC4469557FB551FE52F6FC4242F269558
:1014700090FA9794E92D69C4242F269580FA8794D1
:10148000E82D63C4242F2695B0FAB794EB2D5DC4E4
:10149000242F2695A0FAA794EA2D57C4242F269529
:1014A00070FB7795E72F51C4242F269560FB679535
:1014B000E62F4BC46BD4242F269500FB0795E02F15
:1014C0003AC4242F269550FB5795E52F3EC497FA32
:1014D000990CE92D3AC487FA880CE82D36C4B7FA7E
:1014E000BB0CEB2D32C4A7FAAA0CEA2D2EC477FB55
:1014F000770FE72F2AC467FB660FE62F26C446D472
:1015000007FB000FE02F17C457FB550FE52F1DC435
:10151000292D220F90FA9794E92D17C4282D220F18
:1015200080FA8794E82D11C42B2D220FB0FAB794BE
:10153000EB2D0BC42A2D220FA0FAA794EA2D05C487
:10154000272F220F70FB7795E72FFFC3262F220F3F
:1015500060FB6795E62FF9C319D4202F220F00FBFB
:101560000795E02FE8C3252F220F50FB5795E52F55
:10157000ECC397FA990C9328E92DE7C387FA880CF6
:101580008328E82DE2C3B7FABB0CB328EB2DDDC3EB
:10159000A7FAAA0CA328EA2DD8C377FB770F7329E3
:1015A000E72FD3C367FB660F6329E62FCEC3EED3C5
:1015B00007FB000F0329E02FBEC357FB550F53292C
:1015C000E52FC3C390FA9694E92DBFC380FA8694A1
:1015D000E82DBBC3B0FAB694EB2DB7C3A0FAA6941E
:1015E000EA2DB3C370FB7695E72FAFC360FB66951A
:1015F000E62FABC3CBD300FB0695E02F9CC350FB7B
:101600005695E52FA2C3292D209520FB41F94B7F4C
:101610002EBA40629EC3282D209520FB41F94B7FB6
:101620002EBA406296C32B2D209520FB41F94B7FAB
:101630002EBA40628EC32A2D209520FB41F94B7FA4
:101640002EBA406286C3272F209520FB41F94B7F9D
:101650002EBA40627EC3262F209520FB41F94B7F96
:101660002EBA406276C392D3202F209520FB41F9F9
:101670004B7F2EBA40626DC3252F209520FB41F988
:101680004B7F2EBA406265C3292D209521FB41F97D
:101690004B7F2EBA40625DC3282D209521FB41F976
:1016A0004B7F2EBA406255C32B2D209521FB41F96B
:1016B0004B7F2EBA40624DC32A2D209521FB41F964
:1016C0004B7F2EBA406245C3272F209521FB41F95D
:1016D0004B7F2EBA40623DC3262F209521FB41F956
:1016E0004B7F2EBA406235C351D3202F209521FB6A
:1016F00041F94B7F2EBA40622CC3252F209521FB48
:1017000041F94B7F2EBA406224C3292D209522FB3C
:1017100041F94B7F2EBA40621CC3282D209522FB35
:1017200041F94B7F2EBA406214C32B2D209522FB2A
:1017300041F94B7F2EBA40620CC32A2D209522FB23
:1017400041F94B7F2EBA406204C3272F209522FB1C
:1017500041F94B7F2EBA4062FCC2262F209522FB16
:1017600041F94B7F2EBA4062F4C210D3202F20954E
:1017700022FB41F94B7F2EBA4062EBC2252F209508
:1017800022FB41F94B7F2EBA4062E3C2292D2095FE
:1017900023FB41F94B7F2EBA4062DBC2282D2095F6
:1017A00023FB41F94B7F2EBA4062D3C22B2D2095EB
:1017B00023FB41F94B7F2EBA4062CBC22A2D2095E4
:1017C00023FB41F94B7F2EBA4062C3C2272F2095DD
:1017D00023FB41F94B7F2EBA4062BBC2262F2095D6
:1017E00023FB41F94B7F2EBA4062B3C2CFD2202FE8
:1017F000209523FB41F94B7F2EBA4062AAC2252FC8
:10180000209523FB41F94B7F2EBA4062A2C2292DBD
:10181000209524FB41F94B7F2EBA40629AC2282DB5
:10182000209524FB41F94B7F2EBA406292C22B2DAA
:10183000209524FB41F94B7F2EBA40628AC22A2DA3
:10184000209524FB41F94B7F2EBA406282C2272F9C
:10185000209524FB41F94B7F2EBA40627AC2262F95
:10186000209524FB41F94B7F2EBA406272C28ED282
:10187000202F209524FB41F94B7F2EBA406269C28C
:10188000252F209524FB41F94B7F2EBA406261C27F
:10189000292D209525FB41F94B7F2EBA406259C274
:1018A000282D209525FB41F94B7F2EBA406251C26D
:1018B0002B2D209525FB41F94B7F2EBA406249C262
:1018C0002A2D209525FB41F94B7F2EBA406241C25B
:1018D000272F209525FB41F94B7F2EBA406239C254
:1018E000262F209525FB41F94B7F2EBA406231C24D
:1018F0004DD2202F209525FB41F94B7F2EBA406217
:1019000028C2252F209525FB41F94B7F2EBA406236
:1019100020C2292D209526FB41F94B7F2EBA40622B
:1019200018C2282D209526FB41F94B7F2EBA406224
:1019300010C22B2D209526FB41F94B7F2EBA406219
:1019400008C22A2D209526FB41F94B7F2EBA406212
:1019500000C2272F209526FB41F94B7F2EBA40620B
:10196000F8C1262F209526FB41F94B7F2EBA406205
:10197000F0C10CD2202F209526FB41F94B7F2EBAC7
:101980004062E7C1252F209526FB41F94B7F2EBAF7
:101990004062DFC1292D209527FB41F94B7F2EBAEC
:1019A0004062D7C1282D209527FB41F94B7F2EBAE5
:1019B0004062CFC12B2D209527FB41F94B7F2EBADA
:1019C0004062C7C12A2D209527FB41F94B7F2EBAD3
:1019D0004062BFC1272F209527FB41F94B7F2EBACC
:1019E0004062B7C1262F209527FB41F94B7F2EBAC5
:1019F0004062AFC1CBD1202F209527FB41F94B7F0F
:101A00002EBA4062A6C1252F209527FB41F94B7FB6
:101A10002EBA40629EC12EEF92229BC12EEF8222EF
:101A200098C12EEFB22295C12EEFA22292C12EEFC5
:101A300072238FC12EEF62238CC1A8D12EEF022317
:101A4000AEC12EEF522385C12DEF922282C12DEF20
:101A500082227FC12DEFB2227CC12DEFA22279C15B
:101A60002DEF722376C12DEF622373C18FD12DEF3D
:101A7000022395C12DEF52236CC12BEF922269C135
:101A80002BEF822266C12BEFB22263C12BEFA22281
:101A900060C12BEF72235DC12BEF62235AC176D157
:101AA0002BEF02237CC12BEF522353C127EF92224D
:101AB00050C127EF82224DC127EFB2224AC127EF42
:101AC000A22247C127EF722344C127EF622341C1FD
:101AD0005DD127EF022363C127EF52233AC12FEED6
:101AE000922237C12FEE822234C12FEEB22231C1B1
:101AF0002FEEA2222EC12FEE72232BC12FEE6223D6
:101B000028C144D12FEE02234AC12FEE522321C116
:101B10002FED92221EC12FED82221BC12FEDB2228A
:101B200018C12FEDA22215C12FED722312C12FED86
:101B300062230FC12BD12FED022331C12FED522390
:101B400008C12FEB922205C12FEB822202C12FEB9D
:101B5000B222FFC02FEBA222FCC02FEB7223F9C0F0
:101B60002FEB6223F6C012D12FEB022318C12FEB0B
:101B70005223EFC02FE79222ECC02FE78222E9C068
:101B80002FE7B222E6C02FE7A222E3C02FE772239D
:101B9000E0C02FE76223DDC0F9D02FE70223FFC0AA
:101BA0002FE75223D6C021E0922AD3C021E0822A17
:101BB000D0C021E0B22ACDC021E0A22ACAC021E0D3
:101BC000722BC7C021E0622BC4C0E0D021E0022B01
:101BD000E6C021E0522BBDC022E0922ABAC022E02A
:101BE000822AB7C022E0B22AB4C022E0A22AB1C041
:101BF00022E0722BAEC022E0622BABC0C7D022E045
:101C0000022BCDC022E0522BA4C024E0922AA1C016
:101C100024E0822A9EC024E0B22A9BC024E0A22AAB
:101C200098C024E0722B95C024E0622B92C0AED005
:101C300024E0022BB4C024E0522B8BC028E0922A6F
:101C400088C028E0822A85C028E0B22A82C028E025
:101C5000A22A7FC028E0722B7CC028E0622B79C0CA
:101C600095D028E0022B9BC028E0522B72C020E1C7
:101C7000922A6FC020E1822A6CC020E1B22A69C09A
:101C800020E1A22A66C020E1722B63C020E1622B12
:101C900060C07CD020E1022B82C020E1522B59C0D1
:101CA00020E2922A56C020E2822A53C020E2B22AC1
:101CB00050C020E2A22A4DC020E2722B4AC020E28E
:101CC000622B47C063D020E2022B69C020E2522B76
:101CD00040C020E4922A3DC020E4822A3AC020E499
:101CE000B22A37C020E4A22A34C020E4722B31C0CB
:101CF00020E4622B2EC04AD020E4022B50C020E406
:101D0000522B27C020E8922A24C020E8822A21C032
:101D100020E8B22A1EC020E8A22A1BC020E8722BAD
:101D200018C020E8622B15C031D020E8022B37C044
:101D300020E8522B0EC00ABDE72FF4EBF491E62FFA
:101D4000F7FF0193F7FD0E941A21F6EB44912EBA9A
:101D500040F9EE27E92FF4EBF491E82FF7FF01901B
:101D6000F7FD059097FD06FCE02D0196F5E009943E
:101D7000E92FF4EBF491E82FF7FF0191F7FD0591BE
:101D80000196EBEBF8E0E00FF21D0994E72FF4EB7E
:101D9000F491E62FF7FF0191F7FD059108950ABD33
:101DA000E72FF4EBF491E62FF7FF0193F7FD0E9484
:101DB0001A21CFCF0C94CB020C9446000C94540003
:101DC0000C945F000C9462000C9468000C946E00FC
:101DD0000C9478000C947F000C94DA100C948F0013
:101DE0000C9498000C949B000C94A1000C94A700F8
:101DF0000C94B1000C94B8000C94BD000C94CB0072
:101E00000C94D6000C94D9000C94DF000C94E500DF
:101E10000C94EF000C94F4000C94DF100C94FC0074
:101E20000C9405010C9408010C940E010C941401FF
:101E30000C941E010C9423010C94E4100C94F210E9
:101E40000C9408110C940B110C9411110C94171193
:101E50000C9462010C947C010C9421110C942611B9
:101E60000C9440110C9443110C9449110C944F1193
:101E70000C94B7010C94BB010C94BD010C94CB01E4
:101E80000C94E3010C9459110C9460110C9467119B
:101E90000C940C020C9410020C9475110C94180202
:101EA0000C942E020C9431020C9437020C943D02D7
:101EB0000C9447020C944B020C944C020C944E026E
:101EC0000C9450020C947A110C947C110C947E1199
:101ED0000C9459020C945B020C945D020C945E020B
:101EE0000C9460020C9481110C9483110C94851154
:101EF0000C9469020C946B020C946D020C946F02AA
:101F00000C9470020C9488110C948A110C948C110E
:101F10000C9479020C947B020C947D020C947F0249
:101F20000C9481020C948F110C9491110C949311C8
:101F30000C9489020C9496110C9498110C949A119B
:101F40000C949C110C949E110C949F110C94A11153
:101F50000C94A4110C94A6110C94A8110C94AA1121
:101F60000C94AC110C94AE110C94B0110C94B111F2
:101F70000C94B4110C94B6110C94B8110C94BA11C1
:101F80000C94BC110C94BE110C94C0110C94B702AB
:101F90000C94C2110C94BA020C94BC020C94BE02B4
:101FA0000C94C0020C94C4110C94C6110C94C8116A
:101FB0000C94C9020C9400060C9402060C940406BE
:101FC0000C9406060C94CB110C94CE110C94D111E8
:101FD0000C9416060C9418060C941B060C941E0602
:101FE0000C9421060C94D5110C94D9110C94DD118C
:101FF0000C9435060C9438060C943A060C943C0666
:102000000C943E060C94E2110C94E5110C94E8112A
:102010000C944E060C9450060C9454060C945806DE
:102020000C945C060C94EC110C94F1110C94F611C8
:102030000C9474060C9478060C947A060C947C0626
:102040000C947E060C94FC110C94FF110C9402125B
:102050000C948E060C9490060C9492060C949406A4
:102060000C9496060C9406120C9409120C940C1203
:102070000C94A6060C94A8060C94AA060C94AC0624
:102080000C94AE060C9410120C9413120C941612AD
:102090000C94BE060C94C0060C94C2060C94C406A4
:1020A0000C94C6060C941A120C941D120C94201257
:1020B0000C94D6060C94D8060C94DA060C94EA0616
:1020C0000C94EC060C94FB060C94FD060C9409078A
:1020D0000C9414070C9416070C9418070C941A0708
:1020E0000C9424120C941E070C9420070C942207C5
:1020F0000C942E070C9430070C9432070C94420772
:102100000C9444070C9452070C9454070C946007E9
:102110000C946B070C946D070C946F070C948B0751
:102120000C948D070C949B070C9426120C949F071B
:102130000C94AC070C94AE070C9428120C94C007B6
:102140000C9438120C94D9070C944F120C94E70796
:102150000C94F2070C94F4070C945B120C94F9079E
:102160000C945D120C94FF070C9461120C940308FC
:102170000C940E080C9410080C9412080C9422086D
:102180000C9424080C9425080C9427080C9433080C
:102190000C943E080C9440080C9462120C94450870
:1021A0000C9447080C9448080C9465120C944C0845
:1021B0000C9457084695C80CD91C441F88C14695F5
:1021C000CA0CDB1C441F83C1E92FF4EBF491E82F08
:1021D000F7FFC190F7FDC590F7FFD190F7FDD590BF
:1021E000029676C1E92FF4EBF491E82FF7FFA19165
:1021F000F7FDA591F7FFB191F7FDB5910296EB2F91
:10220000F4EBF491EA2FF7FFC192F7FFD19260C18E
:10221000C30CD21C5DC140FBD30C4FB740F92EBAA2
:1022200057C140FBD3184FB740F93EBA51C1E92F0F
:10223000F4EBF491E82FF7FFD190F7FDD5900196DC
:1022400047C14695CC0CDD1C441F41C1E92FF4EB7E
:10225000F491E82FF7FFA191F7FDA591F7FFB19158
:10226000F7FDB5910296EB2FF4EBF491EA2FF7FF0F
:10227000C190F7FDC590F7FFD190F7FDD59028C12B
:10228000C318D20825C140FBC30C4FB740F92EBA82
:102290001FC140FBC3184FB740F93EBA19C1E92F1F
:1022A000F4EBF491E82FF7FFC190F7FDC59001968C
:1022B0000FC12DD140FB030D4FB740F92EBA4AC1D3
:1022C00026D140FB03194FB740F93EBA43C1E92F6D
:1022D000F4EBF491E82FF7FF1191F7FD1591F7FF5B
:1022E0000191F7FD0591029635C14695C40CD51CA8
:1022F000441FEDC09D2CECC09C2CEAC008D1902E50
:10230000E7C08D2CE5C08C2CE3C001D1802EE0C04D
:10231000BD2CDEC0BC2CDCC0FAD0B02ED9C0AD2C98
:10232000D7C0AC2CD5C0F3D0A02ED2C0D92CD0C0F1
:10233000D82CCEC0DB2CCCC0DA2CCAC0C9C0DC2C57
:10234000C7C0E5D0D02EC4C0D52EC2C0C92CC0C0D5
:10235000C82CBEC0CB2CBCC0CA2CBAC0CD2CB8C0B7
:10236000B7C0D5D0C02EB4C0C52EB2C0092DE9C0AB
:10237000082DE7C00B2DE5C00A2DE3C0072FE1C0F3
:10238000062FDFC0052FDDC05D2DA2C05C2DA0C0D3
:10239000BED0502F9DC05D0D0C94DA025C0D0C94E4
:1023A000DA02B5D0500F0C94DA0246955D1D0C94FC
:1023B000DA0246955C1D0C94DA02A9D04695501FAE
:1023C0000C94DA025D190C94EB025C190C94EB028C
:1023D0009ED0501B0C94EB02469518945D090C940A
:1023E000EB02469518945C090C94EB0290D046954C
:1023F0001894500B0C94EB025D210C9452045C2158
:102400000C94520484D050230C9452045D250C94F7
:1024100065045C250C9465047AD050270C946504FF
:102420005D290C9465045C290C94650470D0502BD4
:102430000C9465045D150C94EB025C150C94EB0296
:1024400066D050170C94EB020C946E1C0C9468121E
:10245000E52DF4EBF491E42DF7FFC190F7FDC59065
:10246000F7FFD190F7FDD590A2E04A0E521C30C084
:10247000D2010601EB2FF4EBF491EA2FF7FFC190A4
:10248000F7FDC590F7FFD190F7FDD590EB2FF4EB5A
:10249000F491EA2FF7FF0192F7FF119219C0A2E021
:1024A0004A1A5208E52DF4EBF491E42DF7FFC1929E
:1024B000F7FFD1920DC0C6010BC0050156016001A6
:1024C00007C006C04C2C5D2C03C00C9468122EBAB9
:1024D000EE27E92FF4EBF491E82FF7FF0190F7FDD9
:1024E000059097FD06FCE02D0196F5E00994E92F93
:1024F000F4EBF491E82FF7FF0191F7FD05910196B8
:10250000EAEDFEE0000FF21DE00FF21D0994E92F45
:10251000F4EBF491E82FF7FF1191F7FD1591019677
:102520000601E12FF0E8EF1B0F1A12080E0E121C25
:10253000E12DF4EBF491E02DF7FF0191F7FD05910A
:102540000895E92FF4EBF491E82FF7FF1191F7FDCF
:10255000159101960601E12FF0E8EF1B0F1A120802
:102560000E0E121C0ABDE12DF4EBF491E02DF7FFE5
:102570000193F7FD0E941A21ABCF0C94CB020C946F
:1025800046000C9454000C945F000C9462000C9470
:1025900068000C94BD140C9478000C947F000C948B
:1025A00089000C948F000C9498000C949B000C9460
:1025B000A1000C94C3140C94B1000C94B8000C94BA
:1025C000BD000C94CB000C94D6000C94D9000C9454
:1025D000DF000C94C9140C94EF000C94F4000C94DC
:1025E000F6000C94FC000C9405010C9408010C946A
:1025F0000E010C94CF140C941E010C9423010C9426
:1026000025010C9433010C9449010C944C010C9459
:1026100052010C94D6140C9462010C947C010C941D
:102620007E010C9484010C949E010C94A1010C94E5
:10263000A7010C94DB140C94B7010C94BB010C940F
:10264000BD010C94CB010C94E3010C94E6010C94B5
:10265000F4010C94E2140C940C020C9410020C94EF
:1026600012020C9418020C942E020C9431020C9459
:1026700037020C94E8140C9447020C944B020C940F
:102680004C020C944E020C9450020C9452020C9486
:1026900054020C94ED140C9459020C945B020C94AB
:1026A0005D020C945E020C9460020C9462020C9425
:1026B00064020C94F6140C9469020C946B020C9452
:1026C0006D020C946F020C9470020C9472020C94C4
:1026D00074020C94FF140C9479020C947B020C94F9
:1026E0007D020C947F020C9481020C9482020C9463
:1026F00084020C9408150C9489020C948B020C949F
:102700008D020C948F020C9491020C9493020C9401
:1027100094020C9411150C9499020C949B020C9445
:102720009D020C949F020C94A1020C94A3020C94A1
:10273000A5020C941A150C94A9020C94AB020C94EB
:10274000AD020C94AF020C94B1020C94B3020C9441
:10275000B5020C9423150C94B8020C94BA020C9494
:10276000BC020C94BE020C94C0020C94C2020C94E5
:10277000C4020C942C150C94C9020C9400060C9401
:1027800002060C9404060C9406060C9408060C949D
:102790000A060C9435150C9416060C9418060C9425
:1027A0001B060C941E060C9421060C9424060C9413
:1027B00027060C9439150C9435060C9438060C94A5
:1027C0003A060C943C060C943E060C9440060C947D
:1027D00042060C943D150C944E060C9450060C9435
:1027E00054060C9458060C945C060C9460060C94E9
:1027F00064060C9441150C9474060C9478060C94A1
:102800007A060C947C060C947E060C9480060C943C
:1028100082060C9445150C948E060C9490060C942C
:1028200092060C9494060C9496060C9498060C94BC
:102830009A060C9449150C94A6060C94A8060C94C0
:10284000AA060C94AC060C94AE060C94B0060C943C
:10285000B2060C944D150C94BE060C94C0060C9454
:10286000C2060C94C4060C94C6060C94C8060C94BC
:10287000CA060C9451150C94D6060C94D8060C94E8
:10288000DA060C94EA060C94EC060C94FB060C9405
:10289000FD060C9455150C9414070C9416070C9413
:1028A00018070C941A070C941C070C941E070C9420
:1028B00020070C9459150C942E070C9430070C9497
:1028C00032070C9442070C9444070C9452070C9462
:1028D00054070C945D150C946B070C946D070C94C5
:1028E0006F070C948B070C948D070C949B070C942A
:1028F0009D070C9461150C94AC070C94AE070C94D6
:10290000B0070C94C0070C94C2070C94D9070C9420
:10291000DB070C9465150C94F2070C94F4070C94E7
:10292000F6070C94F9070C94FB070C94FF070C9422
:1029300001080C9469150C940E080C9410080C9462
:1029400012080C9422080C9424080C9425080C946A
:1029500027080C946D150C943E080C9440080C94B8
:1029600042080C9445080C9447080C9448080C94B1
:102970004A080C9471150C945708D2DD07FB000F20
:1029800000F9E02FB2C0CCDD00FB069507F9E02F7F
:10299000ACC0C6DD469507FB001FE02FA6C0C0DD1A
:1029A000242F269500FB0795E02F9FC0B9DD07FB7C
:1029B000000FE02F9AC0B4DD202F220F00FB0795F7
:1029C000E02F93C0ADDD07FB000F0329E02F8DC082
:1029D000A7DD00FB0695E02F88C0A2DD202F209503
:1029E00020FB41F94B7F2EBA406283C099DD202F36
:1029F000209521FB41F94B7F2EBA40627AC090DDD1
:102A0000202F209522FB41F94B7F2EBA406271C0E6
:102A100087DD202F209523FB41F94B7F2EBA4062A2
:102A200068C07EDD202F209524FB41F94B7F2EBA14
:102A300040625FC075DD202F209525FB41F94B7F5B
:102A40002EBA406256C06CDD202F209526FB41F93E
:102A50004B7F2EBA40624DC063DD202F209527FBAF
:102A600041F94B7F2EBA406244C05ADD2EEF02235B
:102A700071CD56DD2DEF02236DCD52DD2BEF0223FC
:102A800069CD4EDD27EF022365CD4ADD2FEE02230F
:102A900061CD46DD2FED02235DCD42DD2FEB02231C
:102AA00059CD3EDD2FE7022355CD3ADD21E0022B43
:102AB00051CD36DD22E0022B4DCD32DD24E0022B5C
:102AC00049CD2EDD28E0022B45CD2ADD20E1022B69
:102AD00041CD26DD20E2022B3DCD22DD20E4022B7C
:102AE00039CD1EDD20E8022B35CDF6EB44912EBA10
:102AF00040F90601E12FF0E8EF1B0F1A12080E0E45
:102B0000121C0ABDE12DF4EBF491E02DF7FF0193C7
:102B1000F7FD0E941A21EE27E92FF4EBF491E82F3C
:102B2000F7FF0190F7FD059097FD06FCE02D01965B
:102B3000F5E00994E92FF4EBF491E82FF7FF1191F8
:102B4000F7FD1591F7FF0191F7FD05910296F2E16E
:102B5000EDEB000FF21DE00FF21D09940C94CB0277
:102B60000C9446000C9454000C945F000C9462008A
:102B70000C9468000C946E000C9478000C947F0008
:102B80000C94AE170C948F000C9498000C949B003E
:102B90000C94A1000C94A7000C94B1000C94B80004
:102BA0000C94BD000C94CB000C94D6000C94D9006E
:102BB0000C94DF000C94E5000C94EF000C94F400EE
:102BC0000C94B3170C94FC000C9405010C940801B0
:102BD0000C940E010C9414010C941E010C9423010E
:102BE0000C94B8170C94C6170C94DC170C94DF17D0
:102BF0000C94E5170C94EB170C9462010C947C0177
:102C00000C94F5170C94FA170C9414180C941718CC
:102C10000C941D180C9423180C94B7010C94BB0150
:102C20000C94BD010C94CB010C94E3010C942D1871
:102C30000C9434180C943B180C940C020C94100255
:102C40000C9449180C9418020C942E020C94310226
:102C50000C9437020C943D020C9447020C944B02E6
:102C60000C944C020C944E020C9450020C944E188E
:102C70000C9450180C9452180C9459020C945B024A
:102C80000C945D020C945E020C9460020C94551836
:102C90000C9457180C9459180C9469020C946B02FC
:102CA0000C946D020C946F020C9470020C945C18DE
:102CB0000C945E180C9460180C9479020C947B02AE
:102CC0000C947D020C947F020C9481020C94631886
:102CD0000C9465180C9467180C9489020C946A186B
:102CE0000C946C180C946E180C9470180C94721848
:102CF0000C9473180C9475180C9478180C947A181A
:102D00000C947C180C947E180C9480180C948218E7
:102D10000C9484180C9485180C9488180C948A18B8
:102D20000C948C180C948E180C9490180C94921887
:102D30000C9494180C94B7020C9496180C94BA0244
:102D40000C94BC020C94BE020C94C0020C94981813
:102D50000C949A180C949C180C94C9020C940006BC
:102D60000C9402060C9404060C9406060C949F180E
:102D70000C94A2180C94A5180C9416060C94180622
:102D80000C941B060C941E060C9421060C94A91896
:102D90000C94AD180C94B1180C9435060C943806AC
:102DA0000C943A060C943C060C943E060C94B6180F
:102DB0000C94B9180C94BC180C944E060C94500644
:102DC0000C9454060C9458060C945C060C94C01891
:102DD0000C94C5180C94CA180C9474060C947806BC
:102DE0000C947A060C947C060C947E060C94D018F5
:102DF0000C94D3180C94D6180C948E060C94900650
:102E00000C9492060C9494060C9496060C94DA1882
:102E10000C94DD180C94E0180C94A6060C94A806EB
:102E20000C94AA060C94AC060C94AE060C94E41810
:102E30000C94E7180C94EA180C94BE060C94C00687
:102E40000C94C2060C94C4060C94C6060C94EE189E
:102E50000C94F1180C94F4180C94D6060C94D80623
:102E60000C94DA060C94EA060C94EC060C94FB061F
:102E70000C94FD060C9409070C9414070C94160787
:102E80000C9418070C941A070C94F8180C941E074D
:102E90000C9420070C9422070C942E070C943007F6
:102EA0000C9432070C9442070C9444070C9452077C
:102EB0000C9454070C9460070C946B070C946D07EA
:102EC0000C946F070C948B070C948D070C949B0744
:102ED0000C94FA180C949F070C94AC070C94AE0752
:102EE0000C94FC180C94C0070C940C190C94D90782
:102EF0000C9423190C94E7070C94F2070C94F40734
:102F00000C942F190C94F9070C9431190C94FF07A9
:102F10000C9435190C9403080C940E080C941008AA
:102F20000C9412080C9422080C9424080C94250884
:102F30000C9427080C9433080C943E080C94400819
:102F40000C9436190C9445080C9447080C944808C6
:102F50000C9439190C944C080C9457084695E80CBD
:102F6000F91C441F88C14695EA0CFB1C441F83C111
:102F7000E92FF4EBF491E82FF7FFE190F7FDE590EE
:102F8000F7FFF190F7FDF590029676C1E92FF4EB8B
:102F9000F491E82FF7FFA191F7FDA591F7FFB1910B
:102FA000F7FDB5910296EB2FF4EBF491EA2FF7FFC2
:102FB000E192F7FFF19260C1E30CF21C5DC140FBAE
:102FC000F30C4FB740F92EBA57C140FBF3184FB777
:102FD00040F93EBA51C1E92FF4EBF491E82FF7FF25
:102FE000F190F7FDF590019647C14695EE0CFF1C58
:102FF000441F41C1E92FF4EBF491E82FF7FFA191B1
:10300000F7FDA591F7FFB191F7FDB5910296EB2F72
:10301000F4EBF491EA2FF7FFE190F7FDE590F7FF6D
:10302000F190F7FDF59028C1E318F20825C140FBA7
:10303000E30C4FB740F92EBA1FC140FBE3184FB75E
:1030400040F93EBA19C1E92FF4EBF491E82FF7FFEC
:10305000E190F7FDE59001960FC12DD140FB030DE6
:103060004FB740F92EBA4AC126D140FB03194FB7DA
:1030700040F93EBA43C1E92FF4EBF491E82FF7FF92
:103080001191F7FD1591F7FF0191F7FD059102965A
:1030900035C14695E40CF51C441FEDC09F2CECC0D7
:1030A0009E2CEAC008D1902EE7C08F2CE5C08E2C54
:1030B000E3C001D1802EE0C0BF2CDEC0BE2CDCC03E
:1030C000FAD0B02ED9C0AF2CD7C0AE2CD5C0F3D01B
:1030D000A02ED2C0F92CD0C0F82CCEC0FB2CCCC076
:1030E000FA2CCAC0C9C0FE2CC7C0E5D0F02EC4C09F
:1030F000F52EC2C0E92CC0C0E82CBEC0EB2CBCC071
:10310000EA2CBAC0EF2CB8C0B7C0D5D0E02EB4C0FE
:10311000E52EB2C0092DE9C0082DE7C00B2DE5C092
:103120000A2DE3C0072FE1C0062FDFC0052FDDC049
:103130005F2DA2C05E2DA0C0BED0502F9DC05F0DE0
:103140000C94DA025E0D0C94DA02B5D0500F0C9498
:10315000DA0246955F1D0C94DA0246955E1D0C94CA
:10316000DA02A9D04695501F0C94DA025F190C942C
:10317000EB025E190C94EB029ED0501B0C94EB02F8
:10318000469518945F090C94EB02469518945E09D5
:103190000C94EB0290D046951894500B0C94EB02D3
:1031A0005F210C9452045E210C94520484D050236D
:1031B0000C9452045F250C9465045E250C94650400
:1031C0007AD050270C9465045F290C9465045E291D
:1031D0000C94650470D0502B0C9465045F150C940E
:1031E000EB025E150C94EB0266D050170C94EB02C8
:1031F0000C946E1C0C946812E52DF4EBF491E42D04
:10320000F7FFE190F7FDE590F7FFF190F7FDF590FE
:10321000A2E04A0E521C30C0D2010701EB2FF4EBA2
:10322000F491EA2FF7FFE190F7FDE590F7FFF190B9
:10323000F7FDF590EB2FF4EBF491EA2FF7FF0192F5
:10324000F7FF119219C0A2E04A1A5208E52DF4EBDB
:10325000F491E42DF7FFE192F7FFF1920DC0C70161
:103260000BC005015701700107C006C04E2C5F2C32
:1032700003C00C943C192EBAEE27E92FF4EBF4911D
:10328000E82FF7FF0190F7FD059097FD06FCE02D74
:103290000196F5E00994E92FF4EBF491E82FF7FF9C
:1032A0000191F7FD05910196F5E1EEEA000FF21D9F
:1032B000E00FF21D0994E92FF4EBF491E82FF7FFEA
:1032C0001191F7FD159101960701E12FF0E8EF1B31
:1032D0000F1A12080E0E121CE12DF4EBF491E02DE2
:1032E000F7FF0191F7FD05910895E92FF4EBF491B3
:1032F000E82FF7FF1191F7FD159101960701E12FD6
:10330000F0E8EF1B0F1A12080E0E121C0ABDE12D79
:10331000F4EBF491E02DF7FF0193F7FD0E941A21E1
:10332000ABCF0C94CB020C9446000C9454000C943C
:103330005F000C9462000C9468000C94911B0C9438
:1033400078000C947F000C9489000C948F000C94EE
:1033500098000C949B000C94A1000C94971B0C9467
:10336000B1000C94B8000C94BD000C94CB000C94EC
:10337000D6000C94D9000C94DF000C949D1B0C9487
:10338000EF000C94F4000C94F6000C94FC000C94E8
:1033900005010C9408010C940E010C94A31B0C94D1
:1033A0001E010C9423010C9425010C9433010C9400
:1033B00049010C944C010C9452010C94AA1B0C94DE
:1033C00062010C947C010C947E010C9484010C9499
:1033D0009E010C94A1010C94A7010C94AF1B0C94BA
:1033E000B7010C94BB010C94BD010C94CB010C945F
:1033F000E3010C94E6010C94F4010C94B61B0C94BC
:103400000C020C9410020C9412020C9418020C94EE
:103410002E020C9431020C9437020C94BC1B0C94B9
:1034200047020C944B020C944C020C944E020C94E8
:1034300050020C9452020C9454020C94C11B0C9434
:1034400059020C945B020C945D020C945E020C9485
:1034500060020C9462020C9464020C94CA1B0C94DB
:1034600069020C946B020C946D020C946F020C9424
:1034700070020C9472020C9474020C94D31B0C9482
:1034800079020C947B020C947D020C947F020C94C4
:1034900081020C9482020C9484020C94DC1B0C9428
:1034A00089020C948B020C948D020C948F020C9464
:1034B00091020C9493020C9494020C94E51B0C94CE
:1034C00099020C949B020C949D020C949F020C9404
:1034D000A1020C94A3020C94A5020C94EE1B0C9474
:1034E000A9020C94AB020C94AD020C94AF020C94A4
:1034F000B1020C94B3020C94B5020C94F71B0C941B
:10350000B8020C94BA020C94BC020C94BE020C9447
:10351000C0020C94C2020C94C4020C94001C0C94C3
:10352000C9020C9400060C9402060C9404060C9438
:1035300006060C9408060C940A060C94091C0C94BC
:1035400016060C9418060C941B060C941E060C947C
:1035500021060C9424060C9427060C940D1C0C9444
:1035600035060C9438060C943A060C943C060C94E0
:103570003E060C9440060C9442060C94111C0C94CC
:103580004E060C9450060C9454060C9458060C9459
:103590005C060C9460060C9464060C94151C0C9448
:1035A00074060C9478060C947A060C947C060C94A1
:1035B0007E060C9480060C9482060C94191C0C94C4
:1035C0008E060C9490060C9492060C9494060C941F
:1035D00096060C9498060C949A060C941D1C0C9458
:1035E000A6060C94A8060C94AA060C94AC060C949F
:1035F000AE060C94B0060C94B2060C94211C0C94EC
:10360000BE060C94C0060C94C2060C94C4060C941E
:10361000C6060C94C8060C94CA060C94251C0C947F
:10362000D6060C94D8060C94DA060C94EA060C9490
:10363000EC060C94FB060C94FD060C94291C0C94CF
:1036400014070C9416070C9418070C941A070C9482
:103650001C070C941E070C9420070C942D1C0C9432
:103660002E070C9430070C9432070C9442070C94EC
:1036700044070C9452070C9454070C94311C0C947E
:103680006B070C946D070C946F070C948B070C94CC
:103690008D070C949B070C949D070C94351C0C947F
:1036A000AC070C94AE070C94B0070C94C0070C94B4
:1036B000C2070C94D9070C94DB070C94391C0C94AA
:1036C000F2070C94F4070C94F6070C94F9070C9489
:1036D000FB070C94FF070C9401080C943D1C0C9400
:1036E0000E080C9410080C9412080C9422080C94E8
:1036F00024080C9425080C9427080C94411C0C9465
:103700003E080C9440080C9442080C9445080C9414
:1037100047080C9448080C944A080C94451C0C94D7
:103720005708D2DD07FB000F00F9E02FB2C0CCDD57
:1037300000FB069507F9E02FACC0C6DD469507FBF8
:10374000001FE02FA6C0C0DD242F269500FB0795A3
:10375000E02F9FC0B9DD07FB000FE02F9AC0B4DD5A
:10376000202F220F00FB0795E02F93C0ADDD07FB54
:10377000000F0329E02F8DC0A7DD00FB0695E02F89
:1037800088C0A2DD202F209520FB41F94B7F2EBA67
:10379000406283C099DD202F209521FB41F94B7FAA
:1037A0002EBA40627AC090DD202F209522FB41F98D
:1037B0004B7F2EBA406271C087DD202F209523FBFE
:1037C00041F94B7F2EBA406268C07EDD202F2095E4
:1037D00024FB41F94B7F2EBA40625FC075DD202F7C
:1037E000209525FB41F94B7F2EBA406256C06CDD17
:1037F000202F209526FB41F94B7F2EBA40624DC009
:1038000063DD202F209527FB41F94B7F2EBA4062C4
:1038100044C05ADD2EEF022371CD56DD2DEF022379
:103820006DCD52DD2BEF022369CD4EDD27EF022354
:1038300065CD4ADD2FEE022361CD46DD2FED02235B
:103840005DCD42DD2FEB022359CD3EDD2FE7022374
:1038500055CD3ADD21E0022B51CD36DD22E0022BA1
:103860004DCD32DD24E0022B49CD2EDD28E0022BA8
:1038700045CD2ADD20E1022B41CD26DD20E2022BC1
:103880003DCD22DD20E4022B39CD1EDD20E8022BC8
:1038900035CDF6EB44912EBA40F90701E12FF0E85F
:1038A000EF1B0F1A12080E0E121C0ABDE12DF4EBCD
:1038B000F491E02DF7FF0193F7FD0E941A21EE2706
:1038C000E92FF4EBF491E82FF7FF0190F7FD059055
:1038D00097FD06FCE02D0196F5E00994E92FF4EB45
:1038E000F491E82FF7FF1191F7FD1591F7FF019182
:1038F000F7FD05910296F9E1E1E9000FF21DE00FF5
:10390000F21D09943EBAEE27E92FF4EBF491E82F6B
:10391000F7FF0190F7FD059097FD06FCE02D01965D
:10392000F5E00994E92FF4EBF491E82FF7FF01910A
:10393000F7FD05910196FCE1E0EAE00FF21D099424
:103940005CC15BC15AC159C158C157C156C155C1AB
:1039500054C153C152C1F4C02EC130C13BC14DC18D
:103960004CC14BC12EC130C132C147C146C145C156
:1039700044C143C142C141C140C13FC13EC13DC13B
:103980003CC13BC13AC139C138C137C136C135C16B
:1039900034C133C132C131C130C12FC12EC12DC19B
:1039A0002CC12BC12AC129C128C127C126C125C1CB
:1039B00024C123C122C121C120C11FC11EC11DC1FB
:1039C0001DC121C125C12AC13FC142C144C146C157
:1039D00048C14CC150C155C137C16DC10EC16EC186
:1039E00070C174C178C17DC12FC132C190C192C173
:1039F00094C198C19CC1A1C127C15DC1B8C1BBC15F
:103A0000BDC1C1C1C5C1F9C01FC122C1F6C0C6C177
:103A1000E6C1EAC1EEC1F1C017C14DC1EEC0EFC1B0
:103A20000FC2EBC012C217C20FC112C1E6C0E5C07F
:103A300028C22CC230C235C207C13DC1DEC0DDC0C4
:103A4000DCC0DBC0DAC0D9C0D8C0D7C0D6C0D5C0B2
:103A5000D4C0D3C0D2C0D1C0D0C0CFC0CEC0CDC0E2
:103A6000CCC0CBC0CAC0C9C0C8C0C7C0C6C0C5C012
:103A7000C4C0C3C0C2C0C1C0C0C0BFC0BEC0BDC042
:103A80002AC235C247C25BC2B8C0B7C0B6C0B5C053
:103A900069C274C286C29AC2B0C0AFC0AEC0ADC067
:103AA000A8C2B2C2C9C2DBC2A8C0A7C0A6C0A5C076
:103AB000E7C2F1C208C31AC3A0C09FC09EC09DC088
:103AC0009CC09BC09AC099C098C097C096C095C032
:103AD00094C093C092C091C090C08FC08EC08DC062
:103AE0008CC08BC08AC089C088C087C086C085C092
:103AF00084C083C082C081C080C07FC07EC07DC0C2
:103B00007CC07BC07AC079C078C077C076C075C0F1
:103B100074C073C072C071C070C06FC06EC06DC021
:103B20006CC06BC06AC069C068C067C066C065C051
:103B300064C063C062C061C060C05FC05EC05DC081
:103B400077FD29C0C4E3D0E4F894ED2FF4EBF491B1
:103B5000EC2FF7FF6193F7FF71937894C395209250
:103B60000601ED2FF4EBF491EC2FF7FF0191F7FD37
:103B7000059107FDC8CE00910601003091F30FEFCB
:103B80000ABDED2FF4EBF491EC2FF7FF0193F7FD55
:103B90000E941A21B8CE009106010030E1F30FEF28
:103BA0000ABDED2FF4EBF491EC2FF7FF0193F7FD35
:103BB0000E941A21A8CE0E94E05DA5CE0E94A05EC0
:103BC000A2CE0E94AA5D9FCE0E94B45D9CCE0E94B0
:103BD000205F99CEB40120922101209220012092F1
:103BE0001001A0E8CBE3D0E4ED2FF4EBF491EC2F3F
:103BF000F7FFA191F7FDA59186CE85CE94010E9495
:103C00009A20902E80CE9401092D0E94D9207BCE3F
:103C100046951894680979094FB774CEE92FF4EBEB
:103C2000F491E82FF7FFA191F7FDA591F7FFB1916E
:103C3000F7FDB5910296EB2FF4EBF491EA2FF7FF25
:103C40008192F7FF91925FCE51954FB73EBA5BCE0E
:103C500068940C940A042092270155CE50932101B8
:103C600052CE94010E949A20802E4DCE9401082DB0
:103C70000E94D92048CE4695681D791D4FB72EBAAF
:103C800042CEE92FF4EBF491E82FF7FFA191F7FD75
:103C9000A591F7FFB191F7FDB5910296EB2FF4EBEB
:103CA000F491EA2FF7FF8190F7FD8590F7FF91904F
:103CB000F7FD959028CE68940C940A045093200147
:103CC00022CE94010E949A20B02E1DCE94010B2D7D
:103CD0000E94D92018CE469518946A097B094FB7DF
:103CE00011CEE92FF4EBF491E82FF7FFA191F7FD46
:103CF000A591F7FFB191F7FDB5910296EB2FF4EB8B
:103D0000F491EA2FF7FFA192F7FFB192FCCD309228
:103D10002701F9CD50912101F6CD94010E949A20FE
:103D2000A02EF1CD94010A2D0E94D920ECCD46950C
:103D30006A1D7B1D4FB72EBAE6CDE92FF4EBF49147
:103D4000E82FF7FFA191F7FDA591F7FFB191F7FDDE
:103D5000B5910296EB2FF4EBF491EA2FF7FFA190C7
:103D6000F7FDA590F7FFB190F7FDB590CCCD02E03F
:103D700000932701C8CD50912001C5CD94010E9428
:103D80009A20702FC0CD9401072F0E94D920BBCD5F
:103D900046951894660B770B4FB7B4CDE72FF4EB2D
:103DA000F491E62FF7FF0191F7FD0591152F507F54
:103DB000202F2F70522B02950F701F701295012B20
:103DC0000ABDE72FF4EBF491E62FF7FF0193F7FD1F
:103DD0000E941A21E52FF5EB44912EBA94CD94015F
:103DE0000E949A20602F8FCD9401062F0E94D92027
:103DF0008ACD4695661F771F4FB72EBA84CDE72F21
:103E0000F4EBF491E62FF7FF0191F7FD0591152FE3
:103E1000507F202F22952F70522B0295007F1F700C
:103E2000012B0ABDE72FF4EBF491E62FF7FF019386
:103E3000F7FD0E941A21E52FF5EB44912EBA63CDD0
:103E400094010E949A20402F5ECD469518946409F3
:103E500075094FB757CDE92FF4EBF491E82FF7FF31
:103E6000A191F7FDA591F7FFB191F7FDB5910296EC
:103E7000EB2FF4EBF491EA2FF7FF4192F7FF519209
:103E800042CD94010E949A20502F3DCD9401052FE0
:103E90000E94D92038CD4695641D751D4FB72EBAA6
:103EA00032CDE92FF4EBF491E82FF7FFA191F7FD64
:103EB000A591F7FFB191F7FDB5910296EB2FF4EBC9
:103EC000F491EA2FF7FF4190F7FD4590F7FF5190ED
:103ED000F7FD559018CD1BD1630D721DA30CB21CBC
:103EE000477D2EBA8218930809F048600CCDE72F61
:103EF000F4EBF491E62FF7FF0191F7FD05915017D0
:103F00004FB7630D720948603EBA8218930809F4EE
:103F1000477FF9CC94010E949A200ABDE72FF4EB69
:103F2000F491E62FF7FF0193F7FD0E941A21630D2C
:103F3000721D3EBA4D7F931809F44260E4CCE72F1E
:103F4000F4EBF491E62FF7FF0191F7FD0591940151
:103F50000E94D920630D721D3EBA4D7F931809F45B
:103F60004260D1CCD4D063197209A318B208477D3E
:103F70003EBA8218930809F04860C5CCE72FF4EBED
:103F8000F491E62FF7FF0191F7FD059150174FB718
:103F90006319720948603EBA8218930809F4477F92
:103FA000B2CC94010E949A200ABDE72FF4EBF49161
:103FB000E62FF7FF0193F7FD0E941A21631972099A
:103FC0003EBA4D7F931809F442609DCCE72FF4EB85
:103FD000F491E62FF7FF0191F7FD059194010E94FE
:103FE000D920631972093EBA4D7F931809F44260D3
:103FF0008ACC8DD0630D721DA30CB21C831892085D
:10400000C1F7477D2EBA7FCC40FBE72FF4EBF4914C
:10401000E62FF7FF0191F7FD059150174FB740F9D3
:104020004860630D721D8318920841FF71F7092DD6
:10403000082909F4477F66CC94010E949A200ABDA2
:10404000E72FF4EBF491E62FF7FF0193F7FD0E94C1
:104050001A21630D721D931879F7426053CCE72F34
:10406000F4EBF491E62FF7FF0191F7FD0591940130
:104070000E94D920630D721D931889F7426042CCCB
:1040800046D063197209A318B20883189208C1F7C1
:10409000477D2EBA38CC40FBE72FF4EBF491E62FA6
:1040A000F7FF0191F7FD059150174FB740F94860B0
:1040B000631972098318920841FF71F7092D0829C5
:1040C00009F4477F1FCC94010E949A200ABDE72F74
:1040D000F4EBF491E62FF7FF0193F7FD0E941A210C
:1040E00063197209931879F742600CCCE72FF4EB4F
:1040F000F491E62FF7FF0191F7FD059194010E94DD
:10410000D92063197209931889F74260FBCBE72F16
:10411000F4EBF491E62FF7FF0191F7FD05910ABD4D
:10412000EB2DF4EBF491EA2DF7FF0193F7FD0E94DC
:104130001A2108952E3F11F50FEF3F3751F43091BA
:104140000601303A11F40EEF08953D3E11F40EEFE2
:104150000895C5E2D0E4ED2FF4EBF491EC2FF7FFD6
:104160000190F7FD0590201599F4C6E2ED2FF4EBD0
:10417000F491EC2FF7FF0191F7FD05912F3E41F4EB
:1041800009D0333021F00B2F313009F00A2F089578
:104190000FEF089500915801ACE9BCE9045610F006
:1041A000B395FCCF0C590A5010F0A395FCCF0A55DB
:1041B00008952E3F19F43092100108952D3F09F40F
:1041C00008952030D1F42092060130920F01CBE304
:1041D000D0E4ED2FF4EBF491EC2FF7FF3191F7FDE4
:1041E000359130683ABDED2FF4EBF491EC2FF7FFE9
:1041F0003193F7FD0E941A2108952030D1F42092C6
:10420000060120920F01CBE3D0E4ED2FF4EBF49103
:10421000EC2FF7FF3191F7FD35913E7F3ABDED2F41
:10422000F4EBF491EC2FF7FF3193F7FD0E941A2184
:1042300008950895F03C29F4E33619F40AB5009383
:104240005801089500E8A0E0B1E02D920A95E9F741
:10425000A0E0B2E02D92B530E9F7A0E0A1B9A0E06E
:10426000A2B9A0E0A4B9A0E0A5B9A0E0A7B9A0E0D8
:10427000A8B9A0E0AAB9A0E0ABB9AA273299A16079
:104280003499A2603399A460A09311012092C000D8
:10429000A0E1A093C100A6E6A093C200A0911101E5
:1042A000A1FD48C0A0FD2DC0B2ECB0938000B9E1E3
:1042B000B0938100F2E0EBE8F0938700E093860092
:1042C000F8E420928900F0938800FEE120928B00B0
:1042D000F0938A00A4E0A0936F005F982092CD0035
:1042E0002092CC00A8E1A093C900A2ECA093CA0040
:1042F0002092CD002092CC00569A559A53983F9820
:104300000895A0E1A2B9AFEFA1B9B2ECB0938000DB
:10431000B9E1B0938100F5E0ECE6F0938700E0931B
:104320008600F8E420928900F0938800A1E0A09331
:104330006F000895B2ECB0938000B9E1B0938100B2
:10434000F4E0A0FFF4E0F0938700FEEFA0FFF6EFAB
:10435000F093860020928900F4E5F0938800F4E061
:10436000F0938B00F8EDF0938A00A6E0A0936F0025
:104370005F9A569A559A3F9A0895209207010091A4
:1043800007010030E1F30895FAE060FCF5E001C0B8
:10439000FFE0C0E8F2B9AFE4C0B9AA95C0B9E1F74F
:1043A000F0931201BAC0FFE0E0E8F2B9AFE4E0B97F
:1043B000AA95E0B9E1F7FFE2F0931201AEC0FF93D6
:1043C000EF93CF93BF93AF93FFB7FF931498C0E8D9
:1043D000F0911201F2B9630C169A0000C0B9000006
:1043E000C0B900001698F62DF030E9F2F83180F2ED
:1043F000F83D18F0F13F60F201C04FC066246A94A6
:104400007394A0910C02B0910D02BF73BE5F119620
:10441000A0930001B0930101E9E1E0932802E0914B
:104420003402F0913502BF2FC0911001C0FD3197C9
:10443000B078FB2BE0933402F0933502E091060153
:10444000F9E5EE0FFF1FA591B591E0910401E2FDA2
:10445000B160A0932502B0932602AF3F81F0E091B6
:104460003B02E068E0933B02E0910F01E0FF07C0F0
:10447000A0913B02A160A0933B0220920F01E0912A
:104480000601E93E49F4E0910401E2FF05C0E4FFC2
:1044900003C021B80C94000040C0A0913B02A7FFCC
:1044A00073CFFFE0C0E8F2B9A8E0C0B90000C0B91E
:1044B000AA95D9F7A0910001B0910101E62DE8512C
:1044C000E770E730CFB7C1FBF7EBFE0FC0E84F93C3
:1044D0005F93DF9352E4ED91E6FD0DC04491D42F3C
:1044E000D295DF70D2B9C0B94F70C0B942B9C0B966
:1044F0005250C0B981F75B5FFFE0F2B9C0B900006C
:10450000C0B95A95D9F7F0931201DF915F914F919D
:1045100026F4A0930001B09301019CC4FF93EF9394
:10452000CF93BF93AF93FFB7FF93AFE0AA95F1F797
:10453000630C721CE0910E01E8B9789470FC04C021
:10454000F0EC6F1608F47EC0E0911101FBEFE0FF84
:10455000F9ED6F1639F45E98E2FF95C3B2E8B093B7
:10456000800091C3FEEFE0FFFCED6F1639F45E9A18
:10457000E2FF89C3B2ECB093800085C3FBE1E0FFAA
:10458000FBEE6F1621F4E0E8E0930E017CC3F0EF40
:10459000E0FFF0ED6F1619F420920E0174C3F9E3F9
:1045A000E0FFF7E06F1609F06EC366247724E9E1B7
:1045B000E0932802E0913402F0913502BF2FC091C0
:1045C0001001C0FD3197B078FB2BE0933402F093DB
:1045D0003502A0910C02B0910D02BF73BE5F11961F
:1045E000A0930001B0930101E0910601F9E5EE0FFF
:1045F000FF1FA591B591E0910401E2FDB160A09388
:104600002502B0932602AF3F81F0E0913B02E068C3
:10461000E0933B02E0910F01E0FF07C0A0913B0255
:10462000A160A0933B0220920F01E0910601E93EB8
:1046300041F4E0910401E2FF04C0E4FF02C00C94E5
:10464000000021C3A0913B02A7FF1DC3A0918400DD
:10465000A0918500A130B1F7A0918400AE31E0F3C4
:10466000AF3100F0A03200F0A13200F0A23200F031
:104670004F935F93DF93A0910001B0910101E62D6C
:10468000E770F7EBFE0F50E8ED91E6FDEFC2C49145
:10469000E0E1E5BFC8B9DC2FCC0FC8B9CC0FD2958B
:1046A000C8B94C2FCC0FC8B9ED91D8B9DD0F4295E0
:1046B000D8B9C49148B9440F000048B9E6FDD6C244
:1046C000C8B9DC2FCC0FC8B9CC0FD295C8B94C2FC4
:1046D000CC0FC8B9ED91D8B9DD0F4295D8B9C491C6
:1046E00048B9440F000048B9E6FDC0C2C8B9DC2F84
:1046F000CC0FC8B9CC0FD295C8B94C2FCC0FC8B9C4
:10470000ED91D8B9DD0F4295D8B9C49148B9440F9D
:10471000000048B9E6FDAAC2C8B9DC2FCC0FC8B961
:10472000CC0FD295C8B94C2FCC0FC8B9ED91D8B9E0
:10473000DD0F4295D8B9C49148B9440F000048B97B
:10474000E6FD94C2C8B9DC2FCC0FC8B9CC0FD29506
:10475000C8B94C2FCC0FC8B9ED91D8B9DD0F42952F
:10476000D8B9C49148B9440F000048B9E6FD7EC2EB
:10477000C8B9DC2FCC0FC8B9CC0FD295C8B94C2F13
:10478000CC0FC8B9ED91D8B9DD0F4295D8B9C49115
:1047900048B9440F000048B9E6FD68C2C8B9DC2F2B
:1047A000CC0FC8B9CC0FD295C8B94C2FCC0FC8B913
:1047B000ED91D8B9DD0F4295D8B9C49148B9440FED
:1047C000000048B9E6FD52C2C8B9DC2FCC0FC8B909
:1047D000CC0FD295C8B94C2FCC0FC8B9ED91D8B930
:1047E000DD0F4295D8B9C49148B9440F000048B9CB
:1047F000E6FD3CC2C8B9DC2FCC0FC8B9CC0FD295AE
:10480000C8B94C2FCC0FC8B9ED91D8B9DD0F42957E
:10481000D8B9C49148B9440F000048B9E6FD26C292
:10482000C8B9DC2FCC0FC8B9CC0FD295C8B94C2F62
:10483000CC0FC8B9ED91D8B9DD0F4295D8B9C49164
:1048400048B9440F000048B9E6FD10C2C8B9DC2FD2
:10485000CC0FC8B9CC0FD295C8B94C2FCC0FC8B962
:10486000ED91D8B9DD0F4295D8B9C49148B9440F3C
:10487000000048B9E6FDFAC1C8B9DC2FCC0FC8B9B1
:10488000CC0FD295C8B94C2FCC0FC8B9ED91D8B97F
:10489000DD0F4295D8B9C49148B9440F000048B91A
:1048A000E6FDE4C1C8B9DC2FCC0FC8B9CC0FD29556
:1048B000C8B94C2FCC0FC8B9ED91D8B9DD0F4295CE
:1048C000D8B9C49148B9440F000048B9E6FDCEC13B
:1048D000C8B9DC2FCC0FC8B9CC0FD295C8B94C2FB2
:1048E000CC0FC8B9ED91D8B9DD0F4295D8B9C491B4
:1048F00048B9440F000048B9E6FDB8C1C8B9DC2F7B
:10490000CC0FC8B9CC0FD295C8B94C2FCC0FC8B9B1
:10491000ED91D8B9DD0F4295D8B9C49148B9440F8B
:10492000000048B9E6FDA2C1C8B9DC2FCC0FC8B958
:10493000CC0FD295C8B94C2FCC0FC8B9ED91D8B9CE
:10494000DD0F4295D8B9C49148B9440F000048B969
:10495000E6FD8CC1C8B9DC2FCC0FC8B9CC0FD295FD
:10496000C8B94C2FCC0FC8B9ED91D8B9DD0F42951D
:10497000D8B9C49148B9440F000048B9E6FD76C1E2
:10498000C8B9DC2FCC0FC8B9CC0FD295C8B94C2F01
:10499000CC0FC8B9ED91D8B9DD0F4295D8B9C49103
:1049A00048B9440F000048B9E6FD60C1C8B9DC2F22
:1049B000CC0FC8B9CC0FD295C8B94C2FCC0FC8B901
:1049C000ED91D8B9DD0F4295D8B9C49148B9440FDB
:1049D000000048B9E6FD4AC1C8B9DC2FCC0FC8B900
:1049E000CC0FD295C8B94C2FCC0FC8B9ED91D8B91E
:1049F000DD0F4295D8B9C49148B9440F000048B9B9
:104A0000E6FD34C1C8B9DC2FCC0FC8B9CC0FD295A4
:104A1000C8B94C2FCC0FC8B9ED91D8B9DD0F42956C
:104A2000D8B9C49148B9440F000048B9E6FD1EC189
:104A3000C8B9DC2FCC0FC8B9CC0FD295C8B94C2F50
:104A4000CC0FC8B9ED91D8B9DD0F4295D8B9C49152
:104A500048B9440F000048B9E6FD08C1C8B9DC2FC9
:104A6000CC0FC8B9CC0FD295C8B94C2FCC0FC8B950
:104A7000ED91D8B9DD0F4295D8B9C49148B9440F2A
:104A8000000048B9E6FDF2C0C8B9DC2FCC0FC8B9A8
:104A9000CC0FD295C8B94C2FCC0FC8B9ED91D8B96D
:104AA000DD0F4295D8B9C49148B9440F000048B908
:104AB000E6FDDCC0C8B9DC2FCC0FC8B9CC0FD2954D
:104AC000C8B94C2FCC0FC8B9ED91D8B9DD0F4295BC
:104AD000D8B9C49148B9440F000048B9E6FDC6C032
:104AE000C8B9DC2FCC0FC8B9CC0FD295C8B94C2FA0
:104AF000CC0FC8B9ED91D8B9DD0F4295D8B9C491A2
:104B000048B9440F000048B9E6FDB0C0C8B9DC2F71
:104B1000CC0FC8B9CC0FD295C8B94C2FCC0FC8B99F
:104B2000ED91D8B9DD0F4295D8B9C49148B9440F79
:104B3000000048B9E6FD9AC0C8B9DC2FCC0FC8B94F
:104B4000CC0FD295C8B94C2FCC0FC8B9ED91D8B9BC
:104B5000DD0F4295D8B9C49148B9440F000048B957
:104B6000E6FD84C0C8B9DC2FCC0FC8B9CC0FD295F4
:104B7000C8B94C2FCC0FC8B9ED91D8B9DD0F42950B
:104B8000D8B9C49148B9440F000048B9E6FD6EC0D9
:104B9000C8B9DC2FCC0FC8B9CC0FD295C8B94C2FEF
:104BA000CC0FC8B9ED91D8B9DD0F4295D8B9C491F1
:104BB00048B9440F000048B9E6FD58C0C8B9DC2F19
:104BC000CC0FC8B9CC0FD295C8B94C2FCC0FC8B9EF
:104BD000ED91D8B9DD0F4295D8B9C49148B9440FC9
:104BE000000048B9E6FD42C0C8B9DC2FCC0FC8B9F7
:104BF000CC0FD295C8B94C2FCC0FC8B9ED91D8B90C
:104C0000DD0F4295D8B9C49148B9440F000048B9A6
:104C1000E6FD2CC0C8B9DC2FCC0FC8B9CC0FD2959B
:104C2000C8B94C2FCC0FC8B9ED91D8B9DD0F42955A
:104C3000D8B9C49148B9440F000048B9E6FD16C080
:104C4000C8B9DC2FCC0FC8B9CC0FD295C8B94C2F3E
:104C5000CC0FC8B9ED91D8B9DD0F4295D8B9C49140
:104C600048B9440F000048B9E6FD00C058B925BE58
:104C7000E62DE770E73021F4A0930001B093010125
:104C8000DF915F914F91E6C0A73E11F45E98E2C0BC
:104C9000A93E11F45E9ADEC0A73009F0DBC066249D
:104CA0007724E9E1E0932802E0913402F0913502A3
:104CB000BF2FC0911001C0FD3197B078FB2BE0935E
:104CC0003402F0933502A0910C02B0910D02BF7333
:104CD000BE5F1196A0930001B0930101E09106011F
:104CE000F9E5EE0FFF1FA591B591E0910401E2FDFA
:104CF000B160A0932502B0932602AF3F81F0E0910E
:104D00003B02E068E0933B02E0910F01E0FF07C047
:104D1000A0913B02A160A0933B0220920F01E09181
:104D20000601E93E41F4E0910401E2FF04C0E4FF22
:104D300002C00C9400008EC0E0918400E036E0F3E5
:104D4000E13600F0E23600F0E33600F0E43600F041
:104D5000EFEFC8E1C093C900C0E2E093CE00F3E0FA
:104D6000FA95F1F7CA950000FFE3B9F72092C90060
:104D700065C047985F991895FF93EF93CF93BF93C2
:104D8000AF93FFB7FF93630C721CD301B695A79541
:104D9000B0FD06C0A25080F2A03C18F0A23C60F228
:104DA00073CFA0913B02A7FF55C0A0910001B09125
:104DB0000101E62DE450EF70EF30CFB7C1FBC09199
:104DC0008400C435E0F3C53500F0C63500F0C735C2
:104DD00000F0C83500F0E695F7EBFE0FC0E2ED916C
:104DE00000000000E6FD16C0E491C8E1C093C900D0
:104DF000E093CE00CFE1ED91E6FD0AC00000000097
:104E0000E4910000E093CE000000CA95A1F711964E
:104E1000C03069F0F8E1F093C900EFEFE093CE0005
:104E200000000000000000000000CA95F1CFC0E8BB
:104E3000C093CE0000002092C90046F0FF91FFBF52
:104E4000AF91BF91CF91EF91FF911895A093000181
:104E5000B0930101E091C000E7FF48C0E091C600B7
:104E6000A0910401FFEAB491B0FF1BC0A7FF03C0EB
:104E7000209206010BC0F0EBEF77A6FDF395A0FDA5
:104E8000E068E491E0930601E0930701AF71A0931D
:104E90000401FF91FFBFAF91BF91CF91EF91FF91BF
:104EA0001895E7FF0EC0E03F11F4A0681DC0E03E7A
:104EB00041F4A06419C0A6FDE9CFA160A7FDAE7FB3
:104EC000E5CFE231C1F3E935B1F3E43121F4A46077
:104ED000A7FDAB7FDBCFE13121F4A061A7FDAF7E61
:104EE000D5CF20920601AF71A0930401FF91FFBFBF
:104EF000AF91BF91CF91EF91FF911895A0E0B0E0F5
:104F00000000000000001197D9F7B9D0ABE0B0E184
:104F1000A0931301B0931401A0915C01A03071F033
:104F200093D2A0915C01A7FF08952BD1ABE0B2E131
:104F3000A0931301B0931401FFD2089517D0ABE0F2
:104F4000B0E1A0931301B09314017ED20895ADC1D6
:104F5000C7C1CDC101C265C200D0AFEFAEBDADB516
:104F6000A7FFFDCFAEB50895AA27F8CFACE5ACBD3D
:104F7000F3DFF2DF2C98AFE9F1DFF6DFAF3149F470
:104F8000F3DFA452A53028F4A857A0935C01ECDF0E
:104F9000EBDF2C9A08952C98A7EDE0DFE5DF2C9A43
:104FA000A7FFF9CF0895F7DF2C98A3E5D7DFA22F4D
:104FB000D5DFA12FD3DFA02FD1DF2C9A0895EBDF0F
:104FC0002C98A3E5F3CFE7DF2C98A4EDC7DFCCDF67
:104FD000CBDFCADFC9DFC8DFA99323193209D9F7AC
:104FE0002C9A0895D8DF2C98A4E8B8DFBDDFBCDF89
:104FF000BBDFA991B3DF23193209D9F72C9A0895A1
:10500000CADF2C98A4E8AADFAFDFAEDFADDF002453
:10501000A4DF0A94E9F72C9A089500271127980134
:105020002C989ADFBF73B064BEBDBF7398DF3EBDDE
:1050300096DF2EBD94DF1EBD92DF0EBD90DFA5E989
:10504000B83009F4A7E88ADF002487DFAF3F11F406
:105050000A94D9F70895EF93FF93E0E0F0E0AE3FB4
:1050600019F4FF91EF910895319711F076DFF7CFA2
:10507000FF91EF910F900F9030925C01E1C12CBC39
:105080002C9A249A259A279A219A209258012092A4
:105090005C01A3E5ACBDA4E0A0936001B0E12C9A53
:1050A0005CDFBA95E9F7C0E0D1E0B0E0B6DFAF3F32
:1050B00011F0A0FD06C02197C1F720925C012C9A47
:1050C00008950AEA11E022273327B8E0A9DFA2FDFC
:1050D00008C042DF41DFAA3A01F5A0E9A0935C01D4
:1050E00009C0B7E39ADFB1E098DFA2FD39C0A2E8BA
:1050F000A0935C01C0E0D0E8B7E38FDFA0915C0132
:10510000A4FD30E4B1E08CDFA0FF0CC02197A1F733
:1051100002E000935C012C9A0895A4E0A0935C0146
:105120002C9A0895A0915C01A4FF10C0A3E8A0935D
:105130005C01BAE372DF11DFAF930FDF0EDF0DDF2B
:10514000AF91A6FF03C0A4E8A0935C01002712E082
:1051500022273327B0E164DF2C9AA0E5ACBD089587
:10516000C0E0D0E8B1E059DFA0FF07C02197D1F738
:1051700003E000935C012C9A0895A1E8A0935C01E0
:10518000E5CF10E020E031E094E082E002E0100F93
:10519000221D321D019709F446C00027A0915C0131
:1051A000A2FF07C0369527951795012F122F232FA1
:1051B0003327B1E135DF4FDFA0915C01A2FF07C0CB
:1051C000000F111F221F322F212F102F0027BCE0AC
:1051D000C8E4D1E0C2DEA993BA95E1F7BBEFBCDE2B
:1051E000BA95E9F72C9AC8E4D1E0ECE2F2E5BAE02E
:1051F00009901590011451F6BA95D1F7B991E2E4EE
:10520000F8E0B03029F01E1B2F0B3209BA95F9CF08
:1052100002E0100F221D321D10935D0120935E01EC
:1052200030935F01089520925C010895A6BD263D4C
:10523000241DB9A6B5AA452F42954F70445E0E9421
:10524000675C452F4F70445E0E94675C0895209212
:105250005B0110915D0120915E0130915F01A09191
:105260005801B2E4AB9F100D211D321DB8E0AB9F79
:10527000200D311DA0915901AF71B2E4AB9F100D0B
:10528000211D321D00915B01000F100F221D321DE8
:105290000027B0915C01B2FF0895369527951795C8
:1052A000012F122F232F33270895C8E4D1E0A091B6
:1052B0005C01A7FF0FC0CBDFB1E1B2DECCDEBCE00A
:1052C0004CDEA993BA95E1F7BBEF46DEBA95E9F754
:1052D0002C9A0895BAE0A6E1A993BA95E9F7089542
:1052E00083D0EF3F21F4ABE1A09300020895E09357
:1052F0005901ADDFC8E4D1E0B1E192DEACDEBCE043
:105300002CDEA993BA95E1F7BBEF26DEBA95E9F753
:10531000E0915201F0915301C9E0D2E020925B018B
:10532000A0915B01A395A0935B0193DFB1E178DECF
:1053300092DE0024A2E01A2E10DEE215F20511F032
:10534000A993319703181208B9F706DE2C9AE215D3
:10535000F20509F0E5CF089547D0EF3F11F00E2F89
:1053600004C0FF3F09F46CC00F2F00935901209235
:105370005B016FDFB8E154DEAEEFF0DDC8E3D1E0F2
:10538000BCE0A991EBDDBA95E1F7BBEFE5DDBA959D
:10539000E9F7E2DDE2DDAF3FE9F72C9AE091420167
:1053A000F0914301C9E0D2E0A0915B01A395A093E5
:1053B0005B014FDFB8E134DEAEEFD0DD0024A2E0C8
:1053C0001A2EAFEFE215F20511F0A9913197C6DD63
:1053D00003181208B1F7C0DDC0DDAF3FE9F72C9A22
:1053E000E215F20509F7B7CF0FE1EFEFFFEF0093FA
:1053F00059015BDFC8E4D1E0A8E3B1E03AE01991DC
:105400001F3F11F4F09159012D91121729F43A958B
:10541000B1F7E0915901089500915901031938F746
:10542000089515DFB8E1FCDDAEEF98DDB0E094DD66
:10543000BA95E9F791DD91DDAF3FE9F72C9A089530
:10544000ACE1A09300020895A0915C01ECEAF4E5C0
:10545000A13029F13A96A13811F13A96A238F9F023
:105460003A96A338E1F03A96A438C9F03A96A838AB
:10547000B1F03A96A93899F03A96AA3881F03A965E
:10548000AB3869F03A96AC3851F03A96A23039F020
:105490003A96A33021F03A96A43009F03A96459115
:1054A000463719F00E94675CFACF089528263729FD
:1054B000002A373700763232281628263729007618
:1054C00038293B1D16282637297638293B1E1628F1
:1054D0002637297638292D28162826372976292B8C
:1054E0003116211D1E300076292B31161D1C1E2061
:1054F0003076292B31161E1C20243076292B3116AC
:10550000201C25223076292B3116241D251E3076AD
:105510002A1626283229201D00762A162832291D0F
:10552000007676762A16283229240076767600339D
:105530003400282637290076A0915C01E6E4F5E5E1
:10554000A7FF3A96ACCF2B3437322639392A297641
:105550003334002B343732263976F89421B8EB01F6
:10556000D250A88113D0A991A7FFFBCFC9E0D2E008
:10557000E0911402F0911502E850F044A99106D090
:105580003197E1F77894AFEFA1B90895B8E0BF93F0
:10559000B4E0A7FDB9E0AA0F299ABF93AF93B2E098
:1055A000ACEE1197F1F700002998B2E0ABEE11973D
:1055B000F1F7AF91BF9100000000BA9569F7B9E12A
:0E55C000ACE51197F1F7BF91BA9509F7089580
:10AF00000101010101012101010101010121810171
:10AF10000100002100110101010121D10101010104
:10AF20002101110101010121D101010101210111C1
:10AF30000101010121D10101010101011101010101
:10AF40000101D1010101010101110101010101C151
:10AF5000010101010101010101000101C101010122
:10AF6000010101010101010001C101010101010013
:10AF70000101010101014101010101010101010082
:10AF80000000004100000000000000000000000080
:10AF900000000000000000000000000000000000B1
:10AFA00000000000000000000000000000000000A1
:10AFB0000000000000000000000000000000000091
:10AFC0000000000000000000000000000000000081
:10AFD0000000000000000000000000000000000071
:10AFE0001000000000000000000000000000000051
:10AFF0002000000000000000000000000000000031
:10B0000000F900F5F3F1F2FC00FAF8F6F4005E0046
:10B01000F7000000007131000000797361773200A1
:10B0200000637864653433000020766674723500FE
:10B03000006E6268677A360000006D6A7537380006
:10B04000002C6B696F303900002E2D6C00705C0095
:10B0500000000000002700000000EA2B0023000091
:10B06000003C00000000EC0000310034370000001C
:10B07000302C32353638EDC3FB2B332D2A39C40042
:10B0800000F900F5F3F1F2FC00FAF8F6F4EB000039
:10B09000F7000000005121000000595341572200E1
:10B0A000004358444524400000A056465452250011
:10B0B000004E4248475A260000004D4A552F2800AE
:10B0C000003B4B494F3D2900003A5F4C00503F0088
:10B0D00000000000006000000000EB2A00270000D4
:10B0E000003E00000000EC0000310034370000009A
:10B0F00030E932353638EDC3FB2B332D2A39C40005
:10B1000044000000000000000000000000000000FB
:10B11000000000000000000000000000000000002F
:10B12000000000000000000000000000000000001F
:10B1300000000000000000C000000000000000C18E
:10B14000000000000000000000002F0000000000D0
:10B1500000000000000000000000EA000000C20043
:10B16000000000000000000000E100E2E00000003C
:10B17000E8E9E500E3E4EDC3FB2BE72D2AE6C40094
:10B18000450000000000000000000000000000007A
:10B19000000000000040000000000000000000006F
:10B1A000000000000000000000000000000000009F
:10B1B000000000000000000000000000007B5B00B9
:10B1C00000000000007D5D000000000000005C0049
:10B1D00000000000000000000000007E00000000F1
:10B1E000007C00000000000000E100E2E000000040
:10B1F000EFEEE500E3E4EDC3FB2BE72D2AE6C40008
:10B20000FFFFFFFFFFFFFFFFFFFFFFFFFFFFFFFF4E
:10B21000FFFFFFFFFFFFFFFFFFFFFFFFFFFFFFFF3E
:10B22000FFFFFFFFFFFFFFFFFFFFFFFFFFFFFFFF2E
:10B23000FFFFFFFFFFFFFFFFFFFFFFFFFFFFFFFF1E
:10B240007FFDF7FCF7FAFFFFF7EEF7DEEFDEFFFF1B
:10B25000EFF6EFFA7FDEBFF67FFABFEE7FFBFEDE92
:10B26000EFFDF7FDF7FBF7F7F7EFF7DFEFDFEFEFB6
:10B27000EFF7EFFBFEFAFEF6FFFFBFFAFFFFFFFF5F
:10B28000F7F6FDFC7FDEFEEEFDF6FBF6FDEEFDDEE5
:10B29000BFDEDFF6BFEEBFF6BFFA7FF67FEEDFFA66
:10B2A000DFFCFBFCFBEEFDFAFBDEDFEEFEDEFBFA75
:10B2B000FEF6FEFADFDEFFFFFFFFFFFFFFFFFFFFEF
:10B2C000FFFFFDFD7FDFFEEFFDF7FBF7FDEFFDDF8D
:10B2D000BFDFDFF7BFEFBFF7BFFB7FF77FEFDFFB1E
:10B2E000DFFDFBFDFBEFFDFBFBDFDFEFFEDFFBFB2D
:10B2F000FEF7FEFBDFDFFFFFFFFFFFFFFFFFFFFFAC
:10B30000FFFFFFFFFFFFFFFFFFFFFFFFFFFFFFFF4D
:10B31000FFFFFFFFFFFFFFFFFFFFFFFFFFFFFFFF3D
:10B32000FFFFFFFFFFFFFFFFFFFFFFFFFFFFFFFF2D
:10B33000FFFFFFFFFFFFFFFFFFFFFFFFFFFFFFFF1D
:10B340007FFCFFFFFFFFFFFFFFFFFFFFFFFFFFFF90
:10B35000FFFFFFFFFFFFFFFFFFFFFFFFFFFFFFFFFD
:10B36000FFFFFFFFFFFFFFFFFFFFFFFFFFFFFFFFED
:10B37000FFFFFFFFFFFFFFFFFFFFFFFFFFFFFFFFDD
:10B38000FFFFFFFFFFFFFFFFFFFFFFFFFFFFFFFFCD
:10B39000FFFFFFFFFFFFFFFFFFFFFFFFFFFFFFFFBD
:10B3A000FFFFFFFFFFFFFFFFFFFFFFFFFFFFFFFFAD
:10B3B000FFFFFFFFFFFFFFFFFFFFFFFFFFFFFFFF9D
:10B3C000FFFFFFFFF7DEEFF6EFEEEFDEFFFFFFFF21
:10B3D000FFFFFFFFBFFDBFFCEFFCFFFFFFFFFFFF15
:10B3E000FFFFFFFFFFFFFFFFFFFFFFFFFFFFFFFF6D
:10B3F000FFFFFFFFFFFFFFFFFFFFFFFFFFFFFFFF5D
:10B40000C0C1C2C3C4C5C6C7C8C9CACBCCCDCECFC4
:10B41000D0D1D2D3D4D5D6D7D8D9DADBDCDDDEDFB4
:10B42000C0C1C2C3C4C5C6C7C8C9CACBCCCDCECFA4
:10B43000D0D1D2D3D4D5D6D7D8D9DADBDCDDDEDF94
:10B4400002030405060708090A0B0C0D0E0F10BFB6
:10B4500002030405060708090A0B0C0D0E0F10BFA6
:10B4600002030405060708090A0B0C0D0E0F10BF96
:10B4700002030405060708090A0B0C0D0E0F10BF86
:10B48000C0C1C2C3C4C5C6C7C8C9CACBCCCDCECF44
:10B49000D0D1D2D3D4D5D6D7D8D9DADBDCDDDEDF34
:10B4A000C0C1C2C3C4C5C6C7C8C9CACBCCCDCECF24
:10B4B000D0D1D2D3D4D5D6D7D8D9DADBDCDDDEDF14
:10B4C00002030405060708090A0B0C0D0E0F10BF36
:10B4D00002030405060708090A0B0C0D0E0F10BF26
:10B4E00002030405060708090A0B0C0D0E0F10BF16
:10B4F00002030405060708090A0B0C0D0E0F10BF06
:10B50000EAE0E0E8E0E8E8E0E0E8E8E0E8E0E0E8F9
:10B51000E0E8E8E0E8E0E0E8E8E0E0E8E0E8E8E0EB
:10B52000E0E8E8E0E8E0E0E8E8E0E0E8E0E8E8E0DB
:10B53000E8E0E0E8E0E8E8E0E0E8E8E0E8E0E0E8CB
:10B54000E0E8E8E0E8E0E0E8E8E0E0E8E0E8E8E0BB
:10B55000E8E0E0E8E0E8E8E0E0E8E8E0E8E0E0E8AB
:10B56000E8E0E0E8E0E8E8E0E0E8E8E0E8E0E0E89B
:10B57000E0E8E8E0E8E0E0E8E8E0E0E8E0E8E8E08B
:10B58000F4FCFCF4FCF4F4FCFCF4F4FCF4FCFCF43B
:10B59000FCF4F4FCF4FCFCF4F4FCFCF4FCF4F4FC2B
:10B5A000FCF4F4FCF4FCFCF4F4FCFCF4FCF4F4FC1B
:10B5B000F4FCFCF4FCF4F4FCFCF4F4FCF4FCFCF40B
:10B5C000FCF4F4FCF4FCFCF4F4FCFCF4FCF4F4FCFB
:10B5D000F4FCFCF4FCF4F4FCFCF4F4FCF4FCFCF4EB
:10B5E000F4FCFCF4FCF4F4FCFCF4F4FCF4FCFCF4DB
:10B5F000FCF4F4FCF4FCFCF4F4FCFCF4FCF4F4FCCB
:10B60000CAC0C0C8C0C8C8C0C0C8C8C0C8C0C0C8F8
:10B61000C0C8C8C0C8C0C0C8C8C0C0C8C0C8C8C0EA
:10B62000C0C8C8C0C8C0C0C8C8C0C0C8C0C8C8C0DA
:10B63000C8C0C0C8C0C8C8C0C0C8C8C0C8C0C0C8CA
:10B64000C0C8C8C0C8C0C0C8C8C0C0C8C0C8C8C0BA
:10B65000C8C0C0C8C0C8C8C0C0C8C8C0C8C0C0C8AA
:10B66000C8C0C0C8C0C8C8C0C0C8C8C0C8C0C0C89A
:10B67000C0C8C8C0C8C0C0C8C8C0C0C8C0C8C8C08A
:10B68000D4DCDCD4DCD4D4DCDCD4D4DCD4DCDCD43A
:10B69000DCD4D4DCD4DCDCD4D4DCDCD4DCD4D4DC2A
:10B6A000DCD4D4DCD4DCDCD4D4DCDCD4DCD4D4DC1A
:10B6B000D4DCDCD4DCD4D4DCDCD4D4DCD4DCDCD40A
:10B6C000DCD4D4DCD4DCDCD4D4DCDCD4DCD4D4DCFA
:10B6D000D4DCDCD4DCD4D4DCDCD4D4DCD4DCDCD4EA
:10B6E000D4DCDCD4DCD4D4DCDCD4D4DCD4DCDCD4DA
:10B6F000DCD4D4DCD4DCDCD4D4DCDCD4DCD4D4DCCA
:10B70000FF0FF000FF0FF00055FF55FFFFFFFFFF99
:10B71000FFFFFFFFFFFFFFFFFFFFFFFFFFFFFFFF39
:10B72000FFFFFFFFFFFFFFFFFFFFFFFFFFFFFFFF29
:10B73000FFFFFFFFFFFFFFFFFFFFFFFFFFFFFFFF19
:10B74000F894D2E0CDE706E70993B8E1A0E2399397
:10B75000AA95E9F70993BA95C9F7ADE7B0E4A093C4
:10B760000C02B0930D02A0ECA0933B0278940895D4
:10B7800000F00FFF00F00FFFAA00AA000000000069
:10B7900000000000000000000000000000000000A9
:10B7A0000000000000000000000000000000000099
:10B7B0000000000000000000000000000000000089
:10B7C000A03210F0AA27B395B83108F0BB27CEE716
:10B7D000D2E001E20B9FC00DD11DCA0FD21D3883EC
:0CB7E000A395A0931301B09314010895E9
:10B80000FF0FF000FF0FF000AAFFAADBE3F7FFC372
:10B81000FBDFFFFFFFFFFFFFFFFFFFFFC3E7C3C328
:10B82000F781C381C3C3C383C3878181C3BDC1FD06
:10B83000BBBFBDBDC383C383C301BDBDBDBD7D81D2
:0AB84000359136FD0895BCDFFBCF03
:10B8800000F00FFF00F00FFF550055241C08003C8E
:10B890000420000000000000000000003C183C3CB8
:10B8A000087E3C7E3C3C3C7C3C787E7E3C423E02BA
:10B8B000444042423C7C3C7C3CFE42424242827ECE
:10B8C00030813F737DDF319137FD0895F9CFAF931C
:10B8D000BF93CF93DF930F933F930F921F92A0914B
:10B8E0001301B0911401342F3F7B6ADF1F900F903A
:0EB8F0003F910F91DF91CF91BF91AF910895DD
:10B90000FF0FF000FF0FF00055FF55DBDDC1FFBD5D
:10B91000F7EFEFFBFFF7FFEBFDEFFFFFB9D7BDBD83
:10B92000E7BFBFFDBDBDBDBDBDBBBFBFBDBDF7FD5D
:10B93000B7BF999DBDBDBDBDBFEFBDBDBDDBBBFBF1
:10B94000F7EBE42FEF7B58E07491709568E03327B4
:10B95000770F379535DF6A95D1F7F395A850B395F2
:0AB960005A9591F7B850A85F0895BA
:10B9800000F00FFF00F00FFFAA00AA24223E0042A1
:10B99000081010040008001402100000462842425B
:10B9A0001840400242424242424440404242080261
:10B9B00048406662424242424010424242244404AD
:10B9C00038E0BEDEA0E0B4E046EABADF4DEBB8DF17
:10B9D00044E2B6DF4DE1B4DFA5E0BDE0E0ECFAEB18
:08B9E0002FDF0E947E272CC01E
:10BA0000FF0FF000FF0FF000AAFFAAFF87D7EFFBA0
:10BA1000F7EFF7F7C1F7FFF7FBFFFFFFB5F7FDF310
:10BA2000D78383FBC3BDBD83BFBD8383BF81F7FDC8
:10BA30008FBFA5ADBDBDBDBDC3EFBDBDBDE7D7F7D4
:10BA40003092100120920601A0EFA09334022092C0
:10BA50003502A0910601A03021F4A0913402A0305B
:06BA6000C1F708950895EE
:10BA800000F00FFF00F00FFF55005500782810045C
:10BA9000081008083E080008040000004A08020CCC
:10BAA000287C7C043C42427C40427C7C407E0802F4
:10BAB00070405A52424242423C10424242182808C8
:10BAC00008003B1C1B1E2000102811002F1B3C34BB
:08BAD000312B3726320008FF7C
:10BB0000FFFFFFFF0F0F0F0F5555FFFFDFC1FFF7BF
:10BB1000F7EFFBEFFFC1C1C1F7FFFFFFADF7C3FDBB
:10BB2000B7FDBDF7BDC181BDBFBDBFBFB1BDF7BDD5
:10BB3000B7BFBDB5BD83AD83FDEFBDBDBDE7EFEFC5
:10BB4000A0915C01A7FD0895ACE1A09300020F90C5
:10BB50000F9008952092590120925A0100270090D9
:10BB600058010E94A727089520925A010091590177
:0CBB70000395009359010E94A727089537
:10BB800000000000F0F0F0F0AAAA0000203E00083B
:10BB900008100410003E3E3E0800000052083C021F
:10BBA00048024208423E7E42404240404E420842E5
:10BBB0004840424A427C527C0210424242181010D5
:10BBC000BFDFC8E3D1E00AE029920A95E9F7E091E6
:10BBD0001402F0911502E950F0443196E993F9937B
:10BBE000FB01FF73FE5FC8E3D1E00081063131F055
:0EBBF000003011F40C94AD2A0AE022C02BC0E4
:10BC0000FFFFFFFF0F0F0F0FAAAAFFFFDFF5FFFFD8
:10BC1000F7EFF7F7C1F7FFF7EFEFF7E79DF7BFBDD6
:10BC200081BDBDEFBDFDBDBDBDBBBFBFBDBDF7BDD2
:10BC3000BBBFBDB9BDBFB5BBBDEFBDDBA5DBEFDF96
:10BC40001191012E1F73199307FC02C00A95C1F7C9
:10BC50000C94AA27319601910F73063269F00C51AA
:10BC60001AE0019F11911F731C51100D103228F41E
:0CBC7000109359010C94AB2727C022C090
:10BC800000000000F0F0F0F055550000200A000020
:10BC9000081008083E080008101008186208404202
:10BCA0007E424210420242424244404042420842E6
:10BCB0004440424642404A44421042245A24102002
:10BCC000ACE1A0930002089501910F730133C1F715
:10BCD00001910F730133A1F7209259010E94AB2704
:10BCE000009159010395003270F700935901F6CF86
:10BD0000FFFFFFFF0F0F0F0F5555FFFF81C1EFF72B
:10BD1000FBDFEFFBFFF7FFEBDFEFF7E7C3C181C30B
:10BD2000F7C3C3EFC3C3BD83C38781BFC3BDC1C353
:10BD3000BD81BDBDC3BFC3BDC3EFC3E7DBBDEF81E5
:10BD4000FFDEC8E3D1E00AE029920A95E9F7F72F70
:10BD5000E62FF7FD11C0FF73FE5FC8E3D1E00AE0F4
:10BD60001191012E1F731D3041F0199307FC02C081
:0CBD70000A95B1F70C94A827089522C092
:10BD800000000000F0F0F0F0AAAA00007E3E1008CB
:10BD90000420100400080014201008183C3E7E3CCB
:10BDA000083C3C103C3C427C3C787E403C423E3C63
:10BDB000427E42423C403C423C103C182442107EB1
:10BDC000019107FD7DCF0C511AE0019F119117FFE2
:10BDD00077CF1F731C51100D1032D0F7012FE12FB8
:10BDE000E09359010E94A7270090480107FE0C9498
:04BDF000A92766CF4A
:10BE0000FFFFFFFF0F0F0F0FAAAAFFFFFFF7FFFFB4
:10BE1000FFFFFFFFFFFFFFFFFFDFEFFFFFFFFFFF62
:10BE2000FFFFFFFFFFFFFFFFFFFFFFFFFFFFFFFF22
:10BE3000FFFFFFFFFFFFFFFFFFFFFFFFFFFFFFFF12
:10BE400000915A01023088F4102F009159015CE9E9
:10BE50000A5010F05395FCCF0A5510FD502F009159
:10BE60005A01039500935A0108950C3098F51091EA
:0ABE70005C0156E117FFF3CF23C079
:10BE800000000000F0F0F0F0555500000008000040
:10BE90000000000000000000002010000000000072
:10BEA0000000000000000000000000000000000092
:10BEB0000000000000000000000000000000000082
:10BEC000C6E4D1E0C00FD21D08813882003410F4DE
:08BED000502FC5CF5527C3CF49
:10BF0000FFFFFFFFFFFFFFFFFFFFFFFFFFFFFFFF41
:10BF1000CD2A0A3EABD73EAED73EB1D73EAAD73EDA
:10BF2000B8D73E80D73EB4D73EB3D73E80D73EB9D0
:10BF3000D73EA6D73EB5D73EAAD73E80D73E01DB37
:10BF4000EFD73E02DBEFD73E03DBEFD73E76D73E9F
:10BF500076D7C5ED120620C50610ED14D710FBEDFF
:10BF600013C110F3C1C90000000000000000000070
:10BF7000FFFFFFFFFFFFFFFFFFFFFFFFFFFFFFFFD1
:10BF8000FFFFFFFFFFFFFFFFFFFFFFFFFFFFFFFFC1
:10BF9000FFFFFFFFFFFFFFFFFFFFFFFFFFFFFFFFB1
:10BFA000FFFFFFFFFFFFFFFFFFFFFFFFFFFFFFFFA1
:10BFB000FFFFFFFFFFFFFFFFFFFFFFFFFFFFFFFF91
:10BFC0002A3440444D2100002B7CB5F5F120F92A9C
:10BFD0003440E5C5E1C1A7ED42E5C1C91234C9004D
:10BFE000FFFFFFFFFFFFFFFFFFFFFFFFFFFFFFFF61
:10BFF000FFFFFFFFFFFFFFFFFFFFFFFFFFFFFFFF51
:10C00000D3FD01FF7FC3CB032A16402218401846F8
:10C01000A7C2F107C3F507FF2A16407EA7C000009C
:10C02000CD490018F7FFFFFFC39D19F1D9E3D9C926
:10C03000C52A1440E5C388140DC24500E105C8CBEC
:10C04000D9ED4FFBE9D1C818F82A16402322164033
:10C050007EFE7FC018F6E16EFD7500ED7B0240CDDF
:10C060000702C3BC14FF083CFA6D00280208C90887
:10C07000F5C5D5E52A0C40CBFC76D3FDDDE93F3D87
:10C08000283B2638292B2C363C2A37391D1E1F20E9
:10C09000211C2524232235342E3A3E7631302F2D93
:10C0A000001B3233270E190F18E3E1E4E5E2C0D993
:10C0B000E0DBDD75DADEDF7277747370710B1110FF
:10C0C0000DDC79141516D80C1A121317CDCEC178C1
:10C0D000CACBCCD1D2C7C8C9CF4078787878787825
:10C0E00078787878C2D3C4D6D578D4C6C5D07878D5
:10C0F00042D741080A098A8981820784060102879A
:10C10000040577788503838B91908D867892959638
:10C11000888F0B8B26B93926A78F283429AA3B266E
:10C12000B1312AB3382EB32834B83926B32638B300
:10C130002628B82639B331B32A3DB52E33B938365F
:10C14000B7382CB32627B8352A2AB03A38B7383949
:10C15000378D282D378D3334B9179734B72633A947
:10C16000139412941392392D2AB339B438392AB55D
:10C170003135372E33B931312E38B9383934B538F5
:10C180003134BC2B2638B9332ABC3828373431B186
:10C19000283433B9292EB2372AB22B34B72C34398C
:10C1A000B42C34383AA72E33353AB9313426A93174
:10C1B0002E38B9312AB935263A38AA332A3DB9354D
:10C1C0003430AA35372E33B9353134B9373AB3382C
:10C1D000263BAA372633A92EAB2831B83A3335315E
:10C1E00034B928312A26B7372A393A37B3283435B3
:10C1F000BE3733A92E33302A3E8D35AE23EB2A14B9
:10C200004037ED52EBD0E1213B407E17AE17D03ED8
:10C210007F080611D3FE10FED3FD08170000CBFEE9
:10C22000F5C5D5E51803CBB6C92A34402B3E7FA40B
:10C23000B57C2003171802463767223440D0CDBBA7
:10C2400002ED4B254022254078C602ED423A2740B8
:10C25000B4B558060B213B40CB862008CB7ECBC61D
:10C26000C80500372127403FCB1010FE467BFEFE5D
:10C270009F061FB6A01F77D3FF2A0C40CBFCCD92A0
:10C2800002ED5F0101193EF5CDB5022BCD9202C33F
:10C290002902DDE1FD4E28FDCB3B7E280C79ED44E3
:10C2A0003C08D3FEE1D1C1F1C93EFC0601CDB50287
:10C2B0002BE3E3DDE9ED4F3EDDFBE92A2540C9FE36
:10C2C000FEED78F601F6E0572FFE019FB0A56F7CDA
:10C2D000A267CB00ED7838ED1FCB141717179FE638
:10C2E00018C61F322840C9FDCB3B7EC876D3FDFD62
:10C2F000CB3BBEC9CF0ECDA80338F9EBED0CC3077D
:10C30000020F302E10FE1B7AB320F4CD1E03CB7E1D
:10C310002328F8210940CD1E03CDFC0118F85E3713
:10C32000CB13C89FE605C6044FD3FF062310FECDEE
:10C33000460F3072061E10FE0D20EEA710FD18E00D
:10C34000CDA803CB12CB0AEBED0DC307020106000B
:10C350003E7FDBFED3FF1F30491717382810F1F15D
:10C36000BAD2E503626BCD4C03CB7A792003BE20B1
:10C37000D6231730F1FD341521094050CD4C0371FF
:10C38000CDFC0118F6D51E94061A1DDBFE17CB7BDB
:10C390007B38F510F5D12004FE5630B23FCB11307A
:10C3A000ADC97AA728BBCF0CCD550F3A014087FA0B
:10C3B0009A0DE1D0E5CDE702CDF813626B0DF809D7
:10C3C000CBFEC9CDE702ED4B04400BED0E3E3F36F0
:10C3D000022BBC20FAA7ED4209233006352803358D
:10C3E00028F32204402A04402B363E2BF92B2B2223
:10C3F00002403E1EED47ED56FD210040FD363B401C
:10C40000217D40220C40061936762310FB22104075
:10C41000CD9A14CDAD14CD0702CD2A0A2A0A40EDDB
:10C420005B2340A7ED52EB300419222340CDD809FD
:10C430002801EBCD3E07FD351E20372A0A40CDD816
:10C44000092A164037ED52212340300BEB7E23EDB5
:10C45000A01218C5210A405E2356E5EB23CDD8096A
:10C46000CDBB05E1FDCB2D6E2008722B7318AACD34
:10C47000AD142A14407EFE7E2008010600CD600A1D
:10C4800018F3FE762320EECD3705CD1F0A2A14407F
:10C49000FD3600FFCD6607FDCB007E20243A22400A
:10C4A000FE18301D3C322240470E01CD1809545D64
:10C4B0007E2BBE20FC23EB3A0540FE4DDC5D0A18C6
:10C4C000C9210000221840213B40D300CB4628FC64
:10C4D000D30100ED4B2540CD4B0FCDBD0730933A36
:10C4E00006403DFA0805200F3206401D7BD627384E
:10C4F000015F21CC00180E7EFE76282FFE40CBFF78
:10C50000381921C70019180D7EFDCB01562007C62A
:10C51000C0FEE630017EFEF0EA2D055FCD37057BDB
:10C52000CD2605C37204CD9B0912C93E785F2182D6
:10C530000419194E2346C52A1440FDCB2D6E201632
:10C54000FDCB01967EFE7FC823CDB40728F6FE26DC
:10C5500038F2FEDE28EAFDCB01D618E8010100C35F
:10C56000600A9F05540476057F05AF05C4050C06D7
:10C570008B05AF05AF05CD93057E367F23180923C4
:10C580007EFE762818367F2B771898CD9305CD5CE4
:10C590000518F62BED5B14401AFE7FC0D118EA2A6D
:10C5A0000A40CDD809EBCDBB05210B40C364047B09
:10C5B000E60732064018E6EB11C2047EE6C020F71B
:10C5C00056235EC9CD1F0A216F04E5FDCB2D6EC039
:10C5D0002A1440220E402121182239402A0A40CD37
:10C5E000D809CDBB057AB3C82BCDA50A234E234667
:10C5F00023ED5B0E403E7F1213E5211D001909ED6E
:10C6000072E1D0EDB0EBD1CDA6141891CD1F0A2167
:10C610007204FDCB2D6E20112A14407EFEFF2806E9
:10C62000CDE208CD2A0A211904E5CDBA0CE1CD37B7
:10C6300005CD5C05CD730A201578B1C2E0060B0B61
:10C64000ED430740FD362202ED5B0C401813FE76E9
:10C650002812ED4B3040CD1809ED5B2940FD362204
:10C6600002DFFE76CA1304FD360180EB222940EB7F
:10C67000CD4D00CDC10CFDCB018E3EC0FD7719CD57
:10C68000A314FDCB2DAEFDCB007E28222A2940A687
:10C69000201C56235EED530740235E235623EB19DF
:10C6A000CD460F38C7210040CB7E2802360CFDCB8B
:10C6B000387ECC7108012101CD18093A0040ED4BBC
:10C6C00007403C280CFE09200103ED432B402001CC
:10C6D0000BCDEB073E18D7CD980ACDAD14C3C104DE
:10C6E000ED430A402A1640EB211304E52A1A40EDD7
:10C6F00052E5C5000000CD2A0AE1CDD8092006CDBB
:10C70000F209CD600AC1793DB0C8C5030303032B0C
:10C71000CD9E09CD0702C1C5132A1A402BEDB82AB8
:10C720000A40EBC1702B712B732B72C9FDCB01CE6C
:10C73000CDA70E78E63F6769220A40CDD8091E00D2
:10C74000CD450718FBED4B0A40CDEA0916922805A6
:10C75000110000CB13FD731E7EFE40C1D0C5CDA5D8
:10C760000A237AD72323221640FDCB01C6ED4B18AE
:10C77000402A1640A7ED4220033EB8D72A16407E35
:10C7800023CDB40722164028E4FE7F2810FE762829
:10C790005DCB772805CD4B0918D3D718D03A064082
:10C7A00006ABA720053A014006B01F1FE60180CD69
:10C7B000F50718B9FE7EC02323232323C91600CB17
:10C7C000289FF6262E05958537CB1938FA0CC048D8
:10C7D0002D2E0120F2217D005F1937C97BA7F818A3
:10C7E00010AF093C38FCED423D28F11E1C83A72800
:10C7F00004FDCB0186D9E5FDCB014E2005CD08080F
:10C800001803CD5108E1D9C957ED4B394079FE21C4
:10C81000281A3E76BA28302A0E40BE7A20200D20F3
:10C820001923220E400E2105ED43394078FDBE222A
:10C830002803A720DD2E04C35800CD9B09EB7723E6
:10C84000220E40FD3539C90E2105FDCB01C6C318A6
:10C8500009FE76281C4F3A3840E67FFE5C6F264082
:10C86000CC7108712CFD7538C916162A0C40231896
:10C87000051601213C40CDE702C5E5AF5FD3FBE1E2
:10C88000CD460F38051FD3FBCF0CDBFB87FADE0844
:10C8900030EEE5D57AFE029FA307A3574E7923FE1B
:10C8A000762824E5CB278787260FCB14836FCB11FF
:10C8B0009FAE4F06087ACB011F67DBFB1F30FB7C66
:10C8C000D3FB10F1E118D5DBFB1F30FB7A0FD3FB54
:10C8D000D11CCB5B28A7C11520A03E04D3FBCD07FC
:10C8E00002C1215C40367606202B360010FB7DCB42
:10C8F000FF323840C93E1790380BFDBE22DA3508AA
:10C900003C473E1F91DAAD0EC6024FFDCB014E28CB
:10C91000073E5D91323840C9ED4339402A104051FD
:10C920003E22914F3E76042BBE20FC10FA23EDB13F
:10C930002B220E4037E015C8C5CD9E09C141626B60
:10C9400036002B10FBEB23220E40C9F5CD750930C4
:10C9500008FDCB01462002AFD70AE63FD70A03877E
:10C9600030F7C1CB78C8FE1A2803FE38D8AFFDCB0C
:10C9700001C6C3F507E5211101CB7F2802E63FFE82
:10C980004330104704CB7E2328FB10F9CB772002DD
:10C99000FE183F444DE1D00AC6E4C9010100E5CDCF
:10C9A000C50EE1CDAD092A1C40EBEDB8C9F5E52176
:10C9B0000C403E095E2356E3A7ED5219E33009D53A
:10C9C000EB09EB722B7323D1233D20E8EBD1F1A7C8
:10C9D000ED52444D0319EBC9E5217D40545DC1CDB5
:10C9E000EA09D0C5CDF209EB18F47EB8C0237E2B3E
:10C9F000B9C9E57EFE403817CB6F281487FA010AC3
:10CA00003F01050030020E1117237E30FB1806236C
:10CA1000234E23462309D1A7ED52444D19EBC9FDFE
:10CA20004622C5CD2C0AC10518020618FDCB018E81
:10CA30000E21C5CD1809C13A0540FE4D3814FDCB75
:10CA40003AFEAFCDF5072A39407DB4E67E20F3C328
:10CA50001809545D2B480600EDB02A1040CD170A86
:10CA6000C5782F47792F4F03CDAD09EBE119D5EDEF
:10CA7000B0E1C92A1440CD4D00DFFDCB2D6EC021A1
:10CA80005D40221C40CD4815CD8A15380421F0D8D0
:10CA900009DA9A0DBFC3BC14D5E5AFCB782020606E
:10CAA000691EFF1808D556235EE5EB1E000118FC31
:10CAB000CDE107019CFFCDE1070EF6CDE1077DCD6D
:10CAC000EB07E1D1C9CDA60DE1C8E9FDCB01CE7ED2
:10CAD000FE76CA840BD61ACE002869FEA7201BE773
:10CAE000CD920DFE1AC29A0DE7CD920DCD4E0BEFF1
:10CAF0000134CDF50BCDF508183DFEA82033E7CD68
:10CB0000920DCD4E0BCD020CC2AD0EE61F4FFDCBEC
:10CB1000014E280AFD9638CBFFC63CD47108FD862D
:10CB200039FE213A3A40DE01CDFA08FDCB01C618A4
:10CB300006CD550FCD550BDFD61ACE002806CD1DDC
:10CB40000DC3840BD48B0BE7FE76C8C3D50ACDA6E4
:10CB50000DC0E118E2CDC50AFDCB0176CCF8132853
:10CB60000AC3DB153E0BD7ED5B184078B10BC81A32
:10CB700013ED531840CB7728EDFEC028E7C5CD4B09
:10CB800009C118E3CDC50A3E76D7C9CDC50AFDCB8C
:10CB900001C6AFD7ED4B394079FDCB014E28053E9C
:10CBA0005DFD96380E11B930020E01CD0B09C9CDCD
:10CBB000F50BED4336403E2B90DAAD0E473E01CBF0
:10CBC0002830023E04CB29300107F5CDF5087E0759
:10CBD000FE1030060F3002EE8F47119E0C3A3040A7
:10CBE00093FAE90BF12FA01802F1B0FE083802EE1B
:10CBF0008FD9D7D9C9CD020C47C5CD020C59C15127
:10CC00004FC9CDCD15DAAD0E0E01C80EFFC9FD46D8
:10CC1000220E21CD1809CD9B097E12FD343A2A0C33
:10CC20004023545DEDB1C35D0A8B8D2D7F81497525
:10CC30005F40422B171F3752450F6D2B442D5A3B37
:10CC40004C450D525A4D156A0114020600810E061C
:10CC5000DE05AB0D0600B50E00DC0C00D80E04148A
:10CC600006DF0605B90D04002E0E05CF0A0100E906
:10CC70000E050914056A0D00C30303AF0E03300748
:10CC8000061A0600920E036C0E05400305F602001C
:10CC90007C0E009A14002A0A061A0600AF0B061A28
:10CCA0000600AF0B000E0C0600320F002B0F002306
:10CCB0000F00690805CB0A03107FFD360101CD7313
:10CCC0000ACDBC1421004036FF212D40CB6E280E2A
:10CCD000FEE37EC26F0DCDA60DC8CF0CCF08DF06D8
:10CCE00000FE76C84FE779D6E1383B4F21290C0981
:10CCF0004E0918032A30407E2322304001F40CC52F
:10CD00004FFE0B300B21160D0600094E09E5DFC959
:10CD1000DFB92012E7C91725530F6B1376CDA60D87
:10CD2000C0C17EFE76C81872FE76CD9C0DBFC1CC08
:10CD30001D0DEB2A30404E2346EBC5C9CD1C11FD1D
:10CD4000362D003008FDCB2DCE2018CF01CCA711F9
:10CD5000FDCB0176200DAFCDA60DC4F813212D40DB
:10CD6000B677EBED432E40221240C9C13A0140F59F
:10CD7000CD550FF1012113FD5601AAE640201BCB32
:10CD80007A20B7189DCD1C11F579F69F3C200BF148
:10CD900018ADCD550FFDCB0176C0CF0B20F4CDA63D
:10CDA0000DC8EFA034C9FDCB017EC9CDA60D280664
:10CDB000EF02341AA7C8C3DE0CFEE02009E7CD92CB
:10CDC0000DCD1D0D1806CD1D0DEFA134EFC00201D4
:10CDD000E00134CD2113221F402B7ECBFE01060043
:10CDE00009073806CB21CD9E0923E5EF020234E185
:10CDF000EB0E0AEDB02A0740EB13732372CD5A0EE7
:10CE0000D0FDCB087EC0FD462ECBB02A29407EE661
:10CE1000C02017C5CDF209C1232323CD4C00DFFE6E
:10CE2000F3EB20EAEBE7EBB820E4222940C9FDCB85
:10CE30002D4EC24B0D2A1240CB7E281C23221F40B0
:10CE4000EFE0E20FC00234CD5A0ED82A1F40110F76
:10CE500000195E2356EB182ECF00EFE1E0E232001E
:10CE600002010333000434A7C93437C9CDA70E78B3
:10CE7000B12004ED4B3440ED433240C92A2B401819
:10CE800005CDA70E60697CFEF03022CDD80922299D
:10CE900040C9CDCD1538162802ED44F5CDA70EF1C9
:10CEA000FDCB007EC802C9CD8A153801C8CF0ACD96
:10CEB000810EC39A142A074023E3E5ED730240CDA7
:10CEC000810E0106002A1C40093808EB21240019B4
:10CED000ED72D82E03C35800E1E37CFE3E2806ED38
:10CEE00073024018A1E3E5CF06FDCB087E2032CDCA
:10CEF000A314212D40CBEECBB63A0140E64001020F
:10CF00000020020E04B677F73676790F0F38053E0B
:10CF10000B122B772B367F2A3940223040E1C37227
:10CF200004CF07CDE702FDCB3BBEC9FDCB3BFEC323
:10CF30000702CDA70E0000006069ED0B00FD36353D
:10CF4000FFCD070218053E7FDBFE1FFDCB3B863E73
:10CF5000FF322740C9DF0600C5FE40202FCDA60DB9
:10CF60002828ED4B3240CD2015EFA10F30371604A5
:10CF70003080410000802E02A1032D34CD8A15EDB2
:10CF80004332407EA72803D61077180DFE42200DAD
:10CF9000CDA60D2804EFA33434E7C38310FE41204F
:10CFA00011CDBB02444D5114C4BD077A8A424FEBE8
:10CFB000183BCDD214386EFE1BCA471001D809FEAB
:10CFC00016285DFE10200FCD4900CD550FFE112013
:10CFD0002ECD49001822FE0B2028CD4900E518036C
:10CFE000CD4900FE0B2014D1A7ED52444D21014044
:10CFF000CBB6CB7EC4C312E7C38810FE7620E1C354
:10D000009A0DD6C438F901EC04FE13281330F0064B
:10D0100010C6D94FFEDC3002CBB1FEEA3802CBB9E4
:10D02000C5E7C3590FFE26381ECD1C11DA4B0DCCB7
:10D03000A7113A0140FEC0384E23ED5B1C40CDF6EF
:10D0400019EB221C401840CDA60D2023CDD914DFAA
:10D05000010600CD9E0923367E23EB2A1C400E05D7
:10D06000A7ED42221C40EDB0EB2BCD4C001814E78D
:10D07000FE7E20FB23ED5B1C40CDF619ED531C40DA
:10D08000221640FDCB01F6DFFE10200CFDCB017611
:10D09000202ACD6312E718F001C300FE12381DD616
:10D0A000163004C60D180EFE03380AD6C2380DFE1F
:10D0B000063009C603814F214C100946D17AB83891
:10D0C0002CA7CA1800C5D5CDA60D28097BE63F4779
:10D0D000EF373418097BFDAE01E640C29A0DD1212D
:10D0E0000140CBF6CB7B2002CBB6C118CFD579FD62
:10D0F000CB01762015E63FC6084FFE102004CBF189
:10D10000180838D7FE172802CBF9C5E7C3590F0610
:10D1100008080A020305050505050506FDCB01F60D
:10D12000DFCDCE14D29A0DE54FE7E5CBA9FE10284E
:10D1300017CBF1FE0D280CCBE9CDD214300ACBB1C0
:10D14000E718F6E7FDCB01B641CDA60D200879E63C
:10D15000E0CBFF4F18342A10407EE67F282AB92002
:10D160001F1787F29511382DD1D5E5231A13A7285B
:10D17000FBBE28F7F680BE20061ACDD2143015E18A
:10D18000C5CDF209EBC118D1CBF8D1DFFE102809CB
:10D19000CBE8180DD1D1D1E5DFCDD2143003E7189B
:10D1A000F8E1CB10CB70C9AF47CB79204BCB7E20B9
:10D1B0000E3C234E234623EBCDC312DFC35A12236A
:10D1C000232346CB71280A0528E8EBDFFE102061F7
:10D1D000EBEB1824E5DFE1FE1A2820CB792852CBAF
:10D1E000712006FE11203CE7C9FE11286CFEDF20ED
:10D1F00032DF2B221640185E210000E5E7E179FEC0
:10D20000C02009DFFE112851FEDF28E5C5E5CDFF6E
:10D2100012E3EBCDDD1238190BCD051309D1C11086
:10D22000B3CB792066E5CB712013424BDFFE11288A
:10D2300002CF02E7E1110500CD051309C9CDFF12A8
:10D24000E3CD0513C10923424BEBCDC212DFFE1122
:10D250002807FE1A20DBCD6312E7FE1028F8FDCB6D
:10D2600001B6C9CDA60DC4F813E7FE112850D5AFFD
:10D27000F5C5110100DFE1FEDF2817F1CDDE12F563
:10D280005059E5DFE1FEDF2809FE11C29A0D626BFD
:10D290001813E5E7E1FE11280CF1CDDE12F5DF6091
:10D2A00069FE1120E6F1E3192BE3A7ED520100001E
:10D2B000380723A7FA3112444DD1FDCB01B6CDA6D4
:10D2C0000DC8AFC5CDEB19C12A1C4077237323725B
:10D2D0002371237023221C40FDCB01B6C9AFD5E5D5
:10D2E000F5CD920DF1CDA60D2812F5CDA70ED17872
:10D2F000B1372805E1E5A7ED427ADE00E1D1C9EBBF
:10D30000235E2356C9CDA60DC8C506107C4D21004D
:10D3100000293806CB1117300419DAD30E10F2C1E8
:10D32000C92A1240FDCB2D4E284401050003237E5F
:10D33000A728FBCDD21438F5FE0DCAC813F7D52A9D
:10D3400012401B79D606473E40280E237EA728FBB5
:10D35000131210F7F680123E802A1240AEE1CDE79C
:10D3600013E5EF0234E1010500A7ED421840FDCBC3
:10D37000017628061106001918E72A1240ED4B2EF7
:10D3800040FDCB2D46203078B1C8E5F7D5C5545DBA
:10D39000233600EDB8E5CDF813E1E3A7ED420930FF
:10D3A00002444DE3EB78B12802EDB0C1D1E1EB7856
:10D3B000B1C8D5EDB0E1C92B2B2B7EE5C5CDCE1381
:10D3C000C1E1030303C3600A3E602A1240AEF5CDFB
:10D3D000F813EB09E5030303F7EBE10B0BC5EDB81D
:10D3E000EBC10B702B71F1F5CDC714F12B772A1A15
:10D3F000402214402B3680C92A1C402B462B4E2B32
:10D40000562B5E2B7E221C40C9CD1C11C29A0DCD1D
:10D41000A60D2008CBB1CDA711CD1D0D3808C5CD67
:10D42000F209CD600AC1CBF90600C5210100CB711C
:10D4300020022E05EBE72640CDDD12DA3112E1C5E0
:10D4400024E56069CD0513EBDFFE1A28E8FE112004
:10D45000BBE7C17968260023232919DAD30ED5C585
:10D46000E5444D2A14402BCD9E092377C10B0B0BAD
:10D4700023712370F12377626B1B3600C1EDB8C1B5
:10D48000702B712B3D20F8C92A1A402BCD9E092301
:10D4900023C1ED431440C1EB23C92A104036802339
:10D4A0002214402A1440221A40221C40C92A144047
:10D4B000367F23367623FD36220218EA215D40228C
:10D4C0001F402A1A4018E2ED5B1440C35D0AFE2695
:10D4D0001802FE1C3FD0FE40C9CD4815FE1B20158A
:10D4E000EFA1C00234E7CD1415380AEFE0A405C05F
:10D4F000040F3418F0FE2AC0FD365DFFE7FE152844
:10D5000007FE162004FD345DE7CD4815EFE000026C
:10D51000183834C9FE1CD8FE263FD8D61C4F06004A
:10D52000FD210040C5EFA034C1369178A7200777D0
:10D53000B1C8414E368935CB21CB1030F9CB38CB31
:10D5400019237023712B2BC9F5EFA034F1CD1415DD
:10D55000D8EF01A4040F34E718F3EF2D32C00227EF
:10D56000A1032D3200222D303340032D32000C0157
:10D5700002013080481896802F040201A4E00004C4
:10D58000042F0205012FDA0234C9CDF813A72005B4
:10D59000474FF5183143594AD6913FCB78F5CBF830
:10D5A00038243CED44FE08380659480600D608A742
:10D5B000577B072807CB38CB191520F9300803789B
:10D5C000B12003F137F5C5EF34C1F179C9CD8A1522
:10D5D000D8F505042803F137C9F1C9EF2D32000B46
:10D5E0002D33000D02343E1CD7C927343E16D7EF29
:10D5F000347ECD1D15EF307800800330EF1A209A6D
:10D60000850424C1303400031838A20F2434216B60
:10D61000403690060A23E5C5EFA42E0134CDCD1582
:10D62000F690C1E17710EE23010800E52B7EFE9015
:10D6300028FAED42E57EC66BF5F1237ECE0027F594
:10D64000E60F77CBFE28F2F1E1060636802B10FBC1
:10D65000EF02E134CDCD152802ED445F1C1CE12B17
:10D660001D7EE60F28F97BD605FE08F28216FEF62F
:10D67000FA8216C6062848FAB21647CDD01610FB15
:10D68000184043CDD016CDC2163E2AD778A7F298BF
:10D6900016ED44473E1618023E15D77806FF04D60D
:10D6A0000A30FBC60A4F78A72803CDEB0779CDEBEC
:10D6B00007C9ED44473E1BD73E1CD710FD18093E55
:10D6C0001CD73534E83E1BD73534E8CDD01618F8D2
:10D6D0007EE60FCDEB072BC97E3600A7C823CB7E95
:10D6E000CBFE2BC8C501050009414F372B7E2FCE3D
:10D6F000007710F879C1C9E5F54E23467723794EB6
:10D70000C5234E2346EB575ED52356235ED5D9D18C
:10D71000E1C1D92356235EF1E1C9A7C8FE21301625
:10D72000C547D9CB2DCB1ACB1BD9CB1ACB1B10F2AB
:10D73000C1D0CD4117C0D9AF2E00575DD91100001F
:10D74000C91CC014C0D91C200114D9C91AA7C813F8
:10D750001AEE80121BD9E5D9D5E5CDD81647EBCD09
:10D76000D8164FB830037841EBF590CDF716CD1AA7
:10D7700017F1E177E5686119D9EBED4AEB7C8D6F24
:10D780001FADD9EBE11F30083E01CD1A1734282315
:10D79000D97DE680D923772B281F7BED443F5F7A24
:10D7A0002FCE0057D97B2FCE005F7A2FCE003007C7
:10D7B0001FD934CA8018D957D9AF186C373534C837
:10D7C00023AECBFE2BC9AFCDBC17D8D9E5D9D5EB4D
:10D7D000CDBC17EB385AE5CDF71678A7ED62D9E541
:10D7E000ED62D906211811300519D9ED5AD9D9CBD6
:10D7F0001CCB1DD9CB1CCB1DD9CB18CB19D9CB1920
:10D800001F10E4EBD9EBD9C1E178812001A73D3F9E
:10D81000173F1FF219183068A73C20083806D9CBEB
:10D820007AD9205C77D978D930157EA73E80280137
:10D83000AFD9A2CD38170777382E23772B182906B2
:10D8400020D9CB7AD9201207CB13CB12D9CB13CB4B
:10D8500012D93528D710EA18D717300CCD41172028
:10D8600007D91680D9342818E523D9D5D9C1781716
:10D87000CB161F77237123722373E1D1D9E1D9C964
:10D88000CF05EBAFCDBC1738F7EBCDBC17D8D9E53A
:10D89000D9D5E5CDF716D9E56069D96168AF06DF5E
:10D8A000181017CB11D9CB11CB10D929D9ED6AD9C2
:10D8B0003810ED52D9ED52D9300F19D9ED5AD9A7F8
:10D8C0001808A7ED52D9ED52D93704FAA218F52855
:10D8D000E15F51D95950F1CB18F1CB18D9C1E1789A
:10D8E00091C310187EFE81300636003E201805D602
:10D8F000A0F0ED44D5EB2B47CB38CB38CB382805FF
:10D9000036002B10FBE6072809473EFFCB2710FC0B
:10D91000A677EBD1C900B00031003000F1490FDA31
:10D92000A234202F1C721AE3194C17C6178218E272
:10D930001DED1AF31A031B031B031B031B031B031D
:10D940001B5517F81A031B031B031B031B031B03A5
:10D950001B621BA01A061CA41B111C491D3E1D6E38
:10D960001DC41DD41D761DA91C5B1C461CDB1DAFF0
:10D970001AAA1ABE1AC51AD51B8F1BD51AF6193743
:10D980001C231CFC19171CDB1ACE1A2B00181DE4D3
:10D9900018E4195A157F1A511A631A451ACD851BB6
:10D9A00078321E40D9E3D9ED531C40D97E23E5A738
:10D9B000F2C21957E6600F0F0F0FC6726F7AE61F9B
:10D9C000180EFE183008D901FBFF545D09D9076F06
:10D9D0001123192600195E235621A719E3D5D9ED85
:10D9E0004B1D40C9F13A1E40D918C3D5E5010500C9
:10D9F000CDC50EE1D1C9CDEB19EDB0C9626BCDEB50
:10DA000019D9E5D9E3C57EE6C007074F0C7EE63F8E
:10DA10002002237EC650123E059123130600EDB06E
:10DA2000C1E3D9E1D947AF05C8121318FAA7C8F561
:10DA3000D5110000CDFE19D1F13D18F24F07078135
:10DA40004F060009C9D52A1F40CD3C1ACDF619E171
:10DA5000C9626BD9E5211519D9CD2D1ACDFE19D979
:10DA6000E1D9C9E5EB2A1F40CD3C1AEBCDF619EB05
:10DA7000E1C906051A4EEB1271231310F7EBC947E3
:10DA8000CDA0192D0FC002A0C22DE004E2C10334C5
:10DA9000CDFC19CDA4190F01C20231EEE10334C946
:10DAA0007EA7C8237EEE80772BC923CBBE2BC9234C
:10DAB0007E2B353437C4E01A2307CB1E2BC9CDA7E4
:10DAC0000E0AC31D15CDA70E212015E5C5C97EA7D9
:10DAD000C83EFF18077EED443F1805AF23AE2B0765
:10DAE000E5060536002310FBE1D03681C91AA7C828
:10DAF0003718ED1AA7C018E81AA7C0D51BAF121B1C
:10DB000012D1C978D608CB5720013D0F3008F5E572
:10DB1000CD721AD1EBF1CB5720070FF5CD4C17186A
:10DB2000330FF5CDF813D5C5CDF813E17CB5E37807
:10DB3000200BB1C12804F13F1816F11813B1280DBC
:10DB40001A96380920ED0B1323E32B18DFC1F1A738
:10DB5000F5EFA034F1F5DCD51ACDCE1AF10FD4D5FE
:10DB60001AC9CDF813D5C5CDF813E1E5D5C50944DB
:10DB70004DF7CDC312C1E178B12802EDB0C1E17813
:10DB8000B12802EDB02A1C4011FBFFE519D1C9CD27
:10DB9000CD15380E200CF5010100F7F112CDC3129E
:10DBA000EBC9CF0A2A1640E5CDF813D503F7E1ED0E
:10DBB000531640D5EDB0EB2B3676FDCB01BECD92A2
:10DBC0000DCD220DE1221640FDCB01FECD550FE11A
:10DBD00022164018B0010100F736762A3940E52EAA
:10DBE000FF2239402A0E40E5ED530E40D5CDDB151E
:10DBF000D12A0E40A7ED52444DE1220E40E12239D8
:10DC000040CDC312EBC9CDF81378B128011AC31D5A
:10DC100015CDF813C32015D9E5211E4035E12004A8
:10DC200023D9C9D95EAFCB7B28012F5719D9C91A7F
:10DC3000A720F0D923D9C9EFC0022DE00524E001C7
:10DC4000C00403E034C9EF2D3200043634C92D3648
:10DC5000C003E0012C0003A10334C9EF30F138AA5E
:10DC60003B29042D24C3032D0FA1038813365865C7
:10DC7000669D786540A26032C9E721F7AF24EB2F9B
:10DC8000B0B014EE7EBB9458F13A7EF8CFE334CDB9
:10DC9000CD1520073803863009CF053807963004A4
:10DCA000ED4477C9EF02A034C9EF2D33000434CF1F
:10DCB00009A002347E3680CD1D15EF3038000301F7
:10DCC0002D30F04CCCCCCD0333000801A10301343E
:10DCD00034EF0130F0317217F80401A203A2032DD2
:10DCE00030322004A2038C11AC140956DAA5593045
:10DCF000C55C90AA9E706F61A1CBDA96A4319FB4E7
:10DD0000E7A0FE5CFCEA1B43CA36EDA79C7E5EF0F2
:10DD10006E238093040F34C9EF30EE22F9836E0432
:10DD20002DA20F24032D0F2D0F2D27A1032D33C05E
:10DD300000040234C9A103013200021834C9EF35CE
:10DD400027A103E00006182F03EF352D2D042D0F1A
:10DD5000A1038614E65C1F0BA38F38EEE91563BBA5
:10DD600023EE920DCDEDF1235D1BEA0434C9EF2DB6
:10DD70001C011D0534C97EFE81380EEFA118010576
:10DD80002D32A3010006182F03EFA0012D2D042D25
:10DD90000FA1038C10B2130E55E48D5839BC5B985B
:10DDA000FD9E003675A0DBE8B46342C4E6B50936D3
:10DDB000BEE936731B5DECD8DE63BEF061A1B30C27
:10DDC000040F34C9EF2D2D04A1031825A10F05213F
:10DDD0002D0F34C9EF1FA3031834C9EF2D2C001EDB
:10DDE000A234EF012D2C0007220434C35B1C022D4A
:10DDF0002C0009A001330006A1010502A134C9FFCE
:10DE00000000000000000000F0F0F0F00000000052
:10DE10000F0F0F0F00000000FFFFFFFF00000000CA
:10DE200000000000F0F0F0F0F0F0F0F0F0F0F0F0B2
:10DE30000F0F0F0FF0F0F0F0FFFFFFFFF0F0F0F02A
:10DE4000AA55AA55AA55AA5500000000AA55AA55D8
:10DE5000AA55AA550000000000242400000000007C
:10DE6000001C227820207E0000083E283E0A3E0842
:10DE70000000001000001000003C420408000800F0
:10DE800000040808080804000020101010102000EA
:10DE90000000100804081000000004081008040026
:10DEA0000000003E003E0000000008083E08080098
:10DEB000000000003E000000000014083E081400AE
:10DEC00000000204081020000000100000101020C4
:10DED00000000000000808100000000000181800F2
:10DEE000003C464A52623C000018280808083E00E0
:10DEF000003C42023C407E00003C420C02423C009E
:10DF000000081828487E0800007E407C02423C0041
:10DF1000003C407C42423C00007E0204081010009D
:10DF2000003C423C42423C00003C42423E023C003B
:10DF3000003C42427E424200007C427C42427C00E5
:10DF4000003C424040423C00007844424244780059
:10DF5000007E407C40407E00007E407C404040008F
:10DF6000003C42404E423C000042427E424242005F
:10DF7000003E080808083E000002020242423C003F
:10DF800000444870484442000040404040407E0009
:10DF90000042665A42424200004262524A464200F1
:10DFA000003C424242423C00007C42427C404000F5
:10DFB000003C4242524A3C00007C42427C444200C7
:10DFC000003C403C02423C0000FE101010101000CB
:10DFD0000042424242423C00004242424224180077
:10DFE00000424242425A24000042241818244200AF
:10DFF0000082442810101000007E040810207E00CB
:00000001FF
